:100000000C94ED040C940A050C940A050C940A0552
:100010000C9401150C940A050C940A050C940A051D
:100020000C940A050C943F060C940A050C94D30614
:100030000C940A050C940A050C940A050C940A0504
:100040000C940A050C940A050C940A050C940A05F4
:100050000C940A050C940A050C940A050C940A05E4
:100060000C940A050C940A052A0C680C7B0CA81148
:10007000A811A811A811A811A811A811A811A811B8
:10008000A811A811A811A811A811A811A811A811A8
:10009000A811A811A811A811A811A811800CA811C5
:1000A000A80CBC0CD70CFF0C2D0D3E0D520D7C0D79
:1000B000A80DA80DB00EB00EB00EB00E270CED0EB0
:1000C000B10DC80DD00FDA0F5B105B105B105B1029
:1000D0005B10A811A811A811A811A811A811A811A6
:1000E000A811EF0F45105B106364696E6F70737534
:1000F00078585B003C656D7074793E20202020208C
:10010000006572726F723A20777269746520616659
:1001100074657220666F726D61740053494F2D458E
:1001200072726F723A2025690053494F3A434D4429
:100130002054696D656F75740053796E6320576143
:1001400069742E2E2E2020200053746F7070656409
:100150002E2E2E202020003E4E65773C2020202091
:10016000202020004572726F7220696E69742046EB
:1001700041543A20257500252E30386C7820252EE4
:1001800030386C78004572726F7220696E69742025
:1001900053443A202575005344524956452E415444
:1001A00052206E6F7420666F756E6400252E327853
:1001B00020252E327820252E327820252E327820C8
:1001C0002563202575006572726F723A206372652F
:1001D000617465206E65772066696C65000F111388
:1001E00015181A1C1E212325325344726976653175
:1001F00033203230323231323034206279204B4277
:1002000072006279204B42722056312E33005344E3
:10021000726976652D4D41580053444D58252E3452
:10022000750053444D58256875004154520054469A
:10023000542D49443A20252E30347800546170659D
:100240002D456D750058313A2025692C2058323AD9
:100250002025692C2059313A2025692C2059323A21
:100260002025690020202020202020202020202060
:100270000025692066696C65732C207061676520B4
:1002800025692F256920202573202020202020206B
:10029000202020202000C50100000000F0001801EF
:1002A00059CE0000FFFF1E01632059010F00A50079
:1002B00050001E0059CE0000FFFF2201BA205F014E
:1002C0000F00CD0050001E0059CE0000FFFF21019D
:1002D0001C2465019000A50050001E0059CE0000AE
:1002E000FFFF200101246B019000CD0050001E0093
:1002F00059CE0000FFFF1F01632070010F002D0089
:100300005A001E0059CE00001F052A013A24770129
:100310000F0055005A001E0059CE00001F0529018C
:100320003A247E010F007D005A001E0059CE0000C5
:100330001F0528013A2485010F00A50046001E0074
:1003400059CE00001F0527013A248A010F00CD0075
:1003500050001E0059CE00001F0526013A249001CE
:100360000F00F5005A001E0059CE00001F052501A0
:100370003A249701A4007D003C001E0059CE0000E5
:10038000FFFF2401EB276B01A400A5003C001E0029
:1003900059CE0000FFFF230163209C01A4002D0023
:1003A0003C001E0059CE0000FFFF3101E021A001FA
:1003B000A40055003C001E0059CE0000FFFF300194
:1003C000CF21A501A4007D003C001E0059CE0000F5
:1003D000FFFF2F0182206B01A400A5003C001E003E
:1003E00059CE0000FFFF2E016320A801A400CD001C
:1003F0003C001E0059CE0000FFFF2D01EB20AD0197
:10040000A400F5003C001E0059CE0000FFFF2C01A7
:10041000E921C5010F002D009600F00059CE000023
:10042000FFFF2B01F026B2010A00C80032001E00B7
:1004300059CE000000003A014820B6010A00280009
:10044000DB001E0059CE000000003901BD20C601AE
:100450000A005000DB001E0059CE000000003801E9
:10046000BD20D6010A007800DB001E0059CE000036
:1004700000003701BD20E6010A00A000DB001E00DD
:1004800059CE000000003601BD20F6015000C80022
:1004900050001E0059CE0000000035015220FC0122
:1004A000B300C80032001E0059CE0000E00734013E
:1004B000BA2000020A00F00032001E00585400006A
:1004C000DFFF3301BA200402B300F00032001E0047
:1004D00059CE00001F003201AC20C5010A001801EE
:1004E000E5003F0100000000000022028226415486
:1004F00052415458434153434F4D42494E4558454C
:10050000584558584644544150494D47424153522A
:10051000454144590000002421E318C318E318049E
:100520002104210000000000000000000000000085
:1005300000000000000421821041084108410861C8
:100540000861084569456982108210A210A210C393
:1005500018042100008210410820002000200041E2
:100560000841084569456941084108610841086139
:1005700008821000008210200020002000200020AF
:100580000041084569456941084108410841084161
:10059000086108A2108210200020002000200041E5
:1005A0000861086108610861086108610861084123
:1005B000086108A210A21041082000200041086133
:1005C000088210FFFFFFFF0000A210A2108210613E
:1005D000088210A210C318610841084108821082E5
:1005E00010FFFF1F001F00FFFF0000E318A2108292
:1005F000108210C318E3188210610861088210FF8E
:10060000FF1F001F001F001F00FFFFC318A2108262
:10061000108210C318E318821082108210A210FFFB
:10062000FF1F001F001F001F00FFFFC318A2106163
:10063000088210C318C318821061088210A210E348
:1006400018FFFF1F001F00FFFF0000A210821061B3
:10065000086108A2108210610841088210C31804C2
:10066000212421FFFFFFFF0000C318A210821041C8
:1006700008610882101F000000200041088210C39A
:1006800018E318E318E318C318C318A2106108612F
:10069000086108610800000000200041086108A20C
:1006A00010C318C318A210A210A210821061084132
:1006B00008610882106108000020002000610882A3
:1006C00010A210A2108210821082106108610861CD
:1006D000088210A210C3186108410841086108820D
:1006E00010A210A21082108210821082108210823A
:1006F00010C318000000000000000000000000000F
:1007000000000000000000000000000000000000E9
:10071000000000000000E5F0780100000200030383
:1007200030100400000500000807020900000A005C
:10073000000C00000D00000F000010000011070069
:1007400012000013000007010000C80010901611ED
:100750002702003200120D00003200130012290A95
:10076000002B0D0000320030000031040432030081
:100770003505043608083707043803033907073CF2
:1007800004053D08086000276101006A0000800040
:1007900000810000820000830000840000850000CA
:1007A00090100092000093030095100197000098AC
:1007B0000000000000000000005F000000070007CC
:1007C00000147F147F14242A7F2A122313086462E2
:1007D00036495522500005030000001C224100004C
:1007E00041221C0014083E081408083E0808005066
:1007F00030000008080808080060600000201008A9
:1008000004023E5149453E00427F40004261514949
:10081000462141454B311814127F10274545453973
:100820003C4A4949300171090503364949493606B0
:100830004949291E003636000000563600000814CB
:10084000224100141414141400412214080201510E
:100850000906324979413E7E1111117E7F4949498D
:10086000363E414141227F4141221C7F4949494155
:100870007F090909013E4149497A7F0808087F003C
:10088000417F41002040413F017F081422417F40C9
:100890004040407F020C027F7F0408107F3E4141B0
:1008A000413E7F090909063E4151215E7F09192910
:1008B00046464949493101017F01013F4040403FDF
:1008C0001F2040201F3F4038403F63140814630737
:1008D000087008076151494543007F414100020407
:1008E0000810200041417F00040201020440404002
:1008F0004040000102040020545454787F4844448E
:10090000383844444420384444487F3854545418B8
:10091000087E09010218A4A4A47C7F0804047800BE
:10092000447D40004080887A007F102844000041C8
:100930007F40007C041804787C0804047838444420
:100940004438FC2424241818242418FC7C080404AB
:10095000084854545420043F4440203C4040207CEC
:100960001C2040201C3C4030403C44281028441CA3
:10097000A0A0A07C4464544C440008364100000010
:100980007F00000041360800100808100878464132
:100990004678FFFFFFFFFF426C6F636B20257520D9
:1009A0002020202000426175643A202575204C6586
:1009B0006E6774683A202575204761703A20257566
:1009C0002020202000456E64202000426C6F636B65
:1009D000202575202F202575200011241FBECFEF64
:1009E000D8E0DEBFCDBF12E0A0E0B1E0E4E6FCE776
:1009F00002C005900D92A830B107D9F726E0A8E013
:100A0000B2E001C01D92A33EB207E1F70E94BD1102
:100A10000C94303E0C9400000F931F939091210290
:100A2000911131C0E0914001F09141012281338167
:100A300094E1899F200D311D1124F9017096A59133
:100A4000B4918C9182FF03C00FE110E002C009E570
:100A50001EEC462FF9013296849190E03296249153
:100A6000622F70E06B5F7F4F0596413029F0423076
:100A700029F400E018EF02C000EE17E021E043E0A7
:100A800050E00E94202B1F910F910895CF93DF9388
:100A900040E050E090E060E3680F71E3E0914001D6
:100AA000F09141010280F381E02D9F01240F351F59
:100AB000F9017096C591D491F901A591B49128815D
:100AC0002B7F2883891302C02460288320E3290F09
:100AD00011962C931197823048F0891303C0119618
:100AE0007C9304C0913011F411966C939F5F4C5E1F
:100AF0005F4F953099F680912102811102C00E94CA
:100B00006423DF91CF910895A0E1B0E0EAE8F5E039
:100B10000C9446356B017C018E010F5F1F4F80E105
:100B2000F80111928A95E9F7C701B601605F7F4F1E
:100B30008F4F9F4F0E94C21E61157105810591055F
:100B400069F126E932E03A8329834601570124E01E
:100B5000B694A794979487942A95D1F79C828B8218
:100B6000F1E0CF16F8E0DF06F2E0EF06F10418F04E
:100B700020E031E002C020E830E03E832D830E9477
:100B8000271780E1F801A4EBB2E001900D928A955D
:100B9000E1F780E00E94E71680E005C086EC91E076
:100BA0000E94F22581E06096ECE00C946235E62F1D
:100BB000F0E0EC54FB4F6AE00E9494348063808341
:100BC000906391830895E4EBF4E08C549B4F119271
:100BD000E817F907E1F708959091B5059F93909173
:100BE000B4059F931F928F93ECEDF5E083811F92E4
:100BF0008F9382811F928F9381811F928F93808127
:100C00001F928F938CEA91E09F938F9388EC95E0ED
:100C10009F938F930E94013888EC95E00E94C8262C
:100C20008DB79EB740960FB6F8949EBF0FBE8DBF8E
:100C3000089580E090E00E94FA29E0E7F0E08081EA
:100C400081608083E1EBF0E080818760808308959C
:100C5000E0E7F0E080818E7F80831092B100809188
:100C60002102E0914001F091410195E0899FE00D62
:100C7000F11D11240190F081E02D099508951F9236
:100C80000F920FB60F921124EF92FF920F931F93C2
:100C90002F933F934F935F936F937F938F939F9384
:100CA000AF93BF93CF93DF93EF93FF9380910802AD
:100CB0008F5F809308028F7309F50E94D337EC0190
:100CC0000E94D3378C0180E090E00E94FA29C8018D
:100CD0006CE271E00E94B434FC01CE0168E770E080
:100CE0000E94B4342EE0E22E22E0F22E00E010E06A
:100CF00028E03CEF42E0BF010E94702CFF91EF9191
:100D0000DF91CF91BF91AF919F918F917F916F9123
:100D10005F914F913F912F911F910F91FF90EF9015
:100D20000F900FBE0F901F9018950F931F938091F7
:100D30000D0281111EC0E091BE05F091BF058689AC
:100D400081FF09C02FE781E397E121508040904067
:100D5000E1F700C000008BE08093810000EE17E017
:100D600021E043E050E065E070E085E090E00E9423
:100D7000202B81E080930D021F910F9108950F9316
:100D80001F931092810010920D0200E010E021E00C
:100D900043E050E065E070E085E090E00E94202BA9
:100DA0001F910F9108951F920F920FB60F92112469
:100DB0002F933F934F935F936F937F938F939F9363
:100DC000AF93BF93EF93FF9380910D02882319F0A7
:100DD0008F5F80930D0280910D02853110F00E948B
:100DE000BF06FF91EF91BF91AF919F918F917F913E
:100DF0006F915F914F913F912F910F900FBE0F9088
:100E00001F901895A0E0B0E0E8E0F7E00C944B35B7
:100E10008CE392E09093BF058093BE0580913802E9
:100E200090913902A0913A02B0913B028093400226
:100E300090934102A0934202B0934302E12CF12C23
:100E400060E0C7010E94DE18882309F45CC004EB4F
:100E500014E0C1E6D0E0F801D1908F01CE010E94EC
:100E6000E83DD8124CC02196F4E00F3B1F0799F7DC
:100E7000E091BE05F091BF0580819181A281B3818F
:100E800080879187A287B387148615861686178672
:100E900020E130E040E050E0BA0180E00E94E61A34
:100EA000C091BE05D091BF0581E08E8B9091B804B2
:100EB0008091B904892B813011F481E28E8B8A896B
:100EC0009B89AC89BD89BC01CD0160517109810943
:100ED00091091E8915FD05C020E830E040E050E092
:100EE00004C020E031E040E050E00E94C834213DE1
:100EF00032404105510580F010681E8B0DC0EFEFA8
:100F0000EE1AFE0A9DCFE091BE05F091BF05168A4C
:100F100087E991E00E94F225CDB7DEB7E7E00C94B7
:100F20006735A7E0B0E0E7E9F7E00C944035809141
:100F3000DD05811155C040E064E070E08CED95E086
:100F40000E94951F823031F489E291E00E94F225DF
:100F50000C94B911AFE7BCE01197F1F700C00000A5
:100F6000359BFECF882309F43BC090910F02992353
:100F7000B1F01F928F938BE191E09F938F9384EB5D
:100F800094E09F938F930E94013884EB94E00E9439
:100F9000C8260F900F900F900F900F900F90809198
:100FA000C205883239F081E09091C105911180E04D
:100FB0008093C1058091C105882361F0E091C2054D
:100FC000EB3018F0E8EEF1E003C0F0E0E352FE4F42
:100FD000849101C088E690E00E94611F0C94B911D1
:100FE0001091DD058091DC059FEC980F943080F422
:100FF0002091C005813319F42093B6051AC090E002
:1010000030E0205D3F4F8217930771F481E00FC0FD
:10101000813711F00C94B91180EB810F843008F006
:10102000FAC380E38093DC058091DC058F708093A8
:10103000B6058091B605482F50E0B8E18B9FF001CE
:101040001124E45CFD4FF093BF05E093BE05968943
:10105000292F297011F40C94B911133509F40AC120
:10106000292F2B7F268B123209F4DCC018F41132A1
:1010700041F000C1103509F4F9C0173509F4F6C084
:10108000F9C08091BD05813019F40091E70501C0D8
:1010900000E093FF29C081E40E947A1F62E0809102
:1010A000B6050E940C050E9495060023C1F08091B0
:1010B000E505811105C060E87EEC82E090E0C2C0E9
:1010C000813041F0E091BE05F091BF0586898460D2
:1010D000868BEDC060E87EE985E090E0B3C060E01B
:1010E00078E681E090E0AEC094FF07C0C12C78E6BE
:1010F000D72EEE24E394F12C07C060E1C62E68E6FB
:10110000D62EEE24E394F12C8330E1F2811111C04C
:1011100088E1849FF001859FF00D1124E45CFD4F70
:1011200082899389A489B589C816D906EA06FB067F
:1011300049F6011103C000E810E002C000E011E030
:101140001092BD05E091BE05F091BF05878980FD35
:10115000B9CF868986FDB6CF83FF03C0877F868B94
:1011600008C081E40E947A1F62E08091B6050E9467
:101170000C0580E091E00E94E305E091BE05F0914E
:10118000BF05868984FF04C0812C912C54011CC0AA
:1011900050E1852E912CA12CB12C16C0E1E0CE1689
:1011A000DE06E104F10420F0C12CD12C7601D394A9
:1011B0009601B501A40181E00E94E61A892B99F0FD
:1011C0008C0C9D1CAE1CBF1CE091BE05F091BF05B0
:1011D000C288D388E488F588C818D908EA08FB08CB
:1011E000E9F680E001C081E0E4EBF4E098012C54E2
:1011F0003B4F9FEF9193E217F307E1F7882379F0D4
:101200001092B4041092B504E091BE05F091BF05B0
:1012100086898460868B81E091E00E94F22540E01F
:10122000B801D8C693FF1FC081E40E947A1F62E014
:101230008091B6050E940C050E94950660E078E05A
:1012400082E090E00E94840581113CCF1091B605A8
:10125000E091BE05F091BF05808991899093DF05EB
:101260008093DE054AC727FF2DCF65CF62E00E943D
:101270000C0526C061E00E940C058091DD059EEA08
:10128000980F923050F4E091BE05F091BF05968919
:1012900093FF16C0833529F413C08E3489F08F3440
:1012A00079F08F3321F48091C205883249F480911E
:1012B0000F02882309F4C6C38EE40E94EC05C2C362
:1012C00081E40E947A1F8091700080FD0E942806B0
:1012D0008091DD05803509F408C158F48E34B1F0F1
:1012E00008F0A0C08F3311F00C94B9118091C205A1
:1012F00029C3833509F45DC2873509F4F6C0823508
:1013000011F00C94B9110E949506EFC0E090BE0553
:10131000F090BF05D70152964D905D906D907C90F6
:10132000559756968C9183FF0BC09091BD059130D7
:1013300009F472C0412C38E6532E66246394712C54
:10134000B82FB074BD8385FF03C000E011E002C078
:1013500000E810E0C12EDD2480E090E0530142015E
:10136000E0E88E2221EE35E03C832B831C013CE03B
:10137000230E311CDC011196BF83AE830E94E83D31
:10138000EB81FC818193FC83EB838E819F81281606
:10139000390681F7FD81F11113C08091E905909123
:1013A000EA05A091EB05B091EC0588159905AA0511
:1013B000BB0531F48091E70590E08C159D0561F146
:1013C000C1012091E105213069F6C092E705009343
:1013D000E8052D81222341F03DE2430E34EB531EFC
:1013E000611C711C0DE710E0D70156968C9185FFAA
:1013F00006C0B0E84B0EB1E05B1E611C711C980189
:1014000040E050E0C301B2010E94C8343093E305CC
:101410002093E4054093E50540E06CE070E081EE48
:1014200095E0DAC56CE070E081EE95E00E94DC1F8B
:1014300081119FC70091BE051091BF05D801569636
:10144000EC915697F091E705E3FF09C0FF2311F0F7
:10145000E06202C0EF7DD8015696EC9342C0209125
:10146000E505822F90E0A0E0B0E09C01AD012F5F88
:101470003F4F4F4F5F4FA091E105B0E00E942D35E7
:101480009B01AC01A091E305B0E0BA2FAA2780919F
:10149000E405A80FB11D0E9438359B01AC01AF2FA8
:1014A000B0E0BA2FAA278091E805A80FB11D0E94CD
:1014B0003835E4FD04C0605F7F4F8F4F9F4FE5FFDD
:1014C00004C06058714081099109F80102891389AB
:1014D00024893589601771078207930711F083E02B
:1014E00001C081E08093BD0523C780E890E09A8326
:1014F00089831092BD05C090DE05D090DF05C11430
:10150000D10409F452C1E091BE05F091BF05E6890E
:10151000E6FD73C0E1FF15C090910E028091B60503
:10152000981731F00E94BF2F8091B60580930E026C
:1015300042E051E0BE016F5F7F4FC6010E9439302B
:101540003DC0F4E0CF16D10458F421E0C21AD1080E
:10155000D694DC2CCC24D794C794E12CF12C1CC05D
:10156000E5FF03C0A0E0B1E002C0A0E8B0E0BA83AC
:10157000A983A60160E070E09A01AB012450310913
:10158000410951090E942D356B017C0130E8C30EE1
:1015900031E0D31EE11CF11CE4FD05C080E1C80E62
:1015A000D11CE11CF11C8091DD0529813A81823535
:1015B00049F4B701A60180E00E94E61A892B09F4DC
:1015C000F4C0F0C0B90184EB94E00E94DC1F8111EB
:1015D000D0C60E949506E091BE05F091BF058789AF
:1015E00080FDE3C029813A81B701A60181E00E9414
:1015F000E61A892B09F4D9C09BC68091DD05823596
:1016000051F060E870E084EB94E00E94DC1F8823D6
:1016100009F4CBC0AEC680E890E00E94E30594E0F8
:10162000C916D104F0F0E090BE05F090BF05F701B7
:1016300082899389A489B589BC01CD0164587F4F03
:101640008F4F9F4F2DE730E040E050E00E94C834BC
:1016500049015A018901F8E6CF16F1E0DF0629F5C4
:1016600074C0C6019695982F8827979587958351C2
:1016700090402091C30577E0972E920E04EB14E082
:101680007C0120E8E20EF11C5C013FEFA31AB30AD3
:101690000E94E83D873009F4892DD8018D938D0192
:1016A000C501AE14BF0481F7BECFB9E6CB16B1E0D9
:1016B000DB0609F04FC060E0F701808991890E9444
:1016C000DE18A4EBB4E080E090E030E22D914FEB27
:1016D000420F4A3120F040ED420F4A3030F4E82FFB
:1016E000F0E0EC54FB4F20838F5F973011F09A307D
:1016F00049F4981738F0E82FF0E0EC54FB4F3083B2
:101700008F5FF7CF9F5F9B3009F7EFEBF4E082919B
:10171000858324E0E43BF207D1F7E4ECF4E084E3D2
:1017200095E08E179F0711F01192FBCF003932E040
:10173000130710F086E401C082E48093B40481E7CB
:1017400091E09093B8048093B7049092B60480928D
:10175000B50424C081E7C81681E0D806F8F09601E8
:10176000ADE7B0E00E941735AB01BC014D52544BC0
:10177000610971092DE730E080E00E94E61A8D379B
:10178000910520F096012F5F3F4F02C020E030E02E
:1017900030933105209332058093330580E890E043
:1017A0009A83898369817A8114C469817A8141E04D
:1017B00011C490910D02911190E19093B404E091C5
:1017C000BE05F091BF05868987FF03C0906890939E
:1017D000B40485FF05C09091B40490629093B40462
:1017E00082FF07C09091B40494609093B4048B7FFF
:1017F000868B878980FF05C08091B40488608093C0
:10180000B404809102018093B50480EE8093B60405
:101810001092B704ADC081E40E947A1FE091DD050B
:10182000EB3D09F48AC01F7088EF95E09093BF05E7
:101830008093BE058E2F90E0FC01E05CF109E0345E
:10184000F10508F085C5EC5CFF4F0C94093500E00C
:1018500010E0B2C280E091E00E94E3058091DE05D5
:101860009091DF0500EC14E06C01A5E1CA0ED11CDB
:101870007C01BFEFEB1AFB0A60E00E94DE188823B0
:10188000D9F0EC14FD0429F48091B404F8018083AC
:1018900013C0A4EBB4E0C8010B96F8012D9121937D
:1018A000E817F907D9F78091B805D8011B968C93F2
:1018B000045F1F4FC701DCCFE4EBF4E08485819324
:1018C000B5E0E53AFB07D1F740E061EF70E082C395
:1018D0008091DE058A3F08F03BC58093C2051092D7
:1018E000C105EFE7FCE03197F1F700C0000083E4A9
:1018F0000E947A1F5FCB8091DE058093C30518C5D7
:1019000083E292E0A4EBB4E04DEC54E0FC012191C1
:10191000CF012D93F4E0AD3CBF07C1F7A8EFB5E0D0
:1019200085EE94E02D91FA012193AF018E179F0768
:10193000C9F740E061E370E04DC3E091BE05F0916E
:10194000BF0586898093B40440E061E070E042C343
:101950006091DE057091DF0580E090E00E945917EC
:101960006093B4047093B5048093B6049093B70465
:1019700040E064E070E02EC364E070E084EB94E04B
:101980000E94DC1F8111F5C46091B4047091B5040C
:101990008091B6049091B7046093C4057093C50517
:1019A0008093C6059093C7050E942717C1C4609114
:1019B000C4057091C5058091C6059091C7050E9428
:1019C00027178FE79CE00197F1F700C0000083E440
:1019D0000E947A1FAFE7BCE01197F1F700C000004A
:1019E00060E072E084EB92E00E94521F182F60E0EA
:1019F00072E084EB92E00E94811F812FB8C4609155
:101A0000C4057091C5058091C6059091C7050E94D7
:101A1000271740E260E072E084EB92E00E94951F9D
:101A2000EFE9FFE03197F1F700C00000882361F093
:101A30006091C4057091C5058091C6059091C70558
:101A40000E9427178EE493C481E40E947A1F80E0ED
:101A50000E94E71681117CC46BC46091DE05662389
:101A600009F466C4E9EEF1E0A4EBB4E080E09491FF
:101A70009D938F5F31966813FACFAAC20E941E17FA
:101A80008091DE05882319F00E9402075FC48FE76A
:101A90009CE00197F1F700C0000083E40E947A1FE8
:101AA0000C9400009091DE05953008F051C4A8E137
:101AB0009A9FF0011124E45CFD4F868983FD02C0EA
:101AC0008E7F01C0867F868BE0914001F0914101BD
:101AD0000280F381E02DB4E19B9FE00DF11D112404
:101AE000859194914CE050E064EF70E003960E9481
:101AF000E3378091C0055BC2E091DE05E53008F078
:101B000027C428E1E29FF0011124E45CFD4F86899F
:101B100080FD08C08EE090E00E94E30540E06EE0AA
:101B200070E058C2F093BF05E093BE0584819581B3
:101B3000A681B7818093FC059093FD05A093FE05D7
:101B4000B093FF05908981899093DE058093DF052E
:101B500060E08091DE059091DF050E94DE18082F7D
:101B60003CC06BE070E08DEE95E00E94DC1F8111BF
:101B700000C48091DF05882309F4DAC31091DE05E3
:101B8000812F806F8093DD051092DF051092DE05B6
:101B9000E090DE05F090DF058091DD05803F08F0E4
:101BA000B5C160E0C7010E94DE18882309F4F2C1C4
:101BB000EDEEF5E0A4EBB4E081918111C1C1119685
:101BC00035E0E83FF307C1F78091DD05803F08F07D
:101BD000BCC183EE8093DD0501E02091B805209320
:101BE000BF048091DD05833E61F4E091BE05F09174
:101BF000BF05808991899093C1048093C0041EE041
:101C0000A7C0853E09F0A3C0A091BE05B091BF0555
:101C100052964D915D916D917C9155974093C00482
:101C20005093C1046093C2047093C3048091B905BA
:101C3000D090BA058093C404D092C5048091BB05AE
:101C40009091BC059093C7048093C604E8ECF4E03F
:101C500086EE94E030E231938E179F07E1F75296BB
:101C60006D917D918D919C915597287119F420E388
:101C70002093D10444EBE42E44E0F42E1AE05AE021
:101C8000852E912CA12CB12C611571058105910532
:101C900051F0A50194010E94C8346063D7015D969C
:101CA0006C93B901CA011150B1E0EB1AF10811119E
:101CB000EBCF8DE28093D7048093DA048AE380939C
:101CC000E0048093E3048D2D869590E08454984F32
:101CD00064E670E00E94A034962F182F6FE1892FE0
:101CE0000E94D70561E2812F0E94D7058091B90536
:101CF0009091BA0525E0969587952A95E1F764E2DB
:101D00008F700E94D7058091B90567E28F710E949C
:101D1000D7058091BC056AE28695869586950E94D6
:101D2000D7058091BB059091BC0535E096958795C8
:101D30003A95E1F76DE28F730E94D7058091BB055C
:101D40008F7160E3880F0E94D70512E301C01CE089
:101D5000011104C082E390E00E94E305612F38C1C5
:101D600061E08091DE059091DF050E94DE1881110F
:101D700006C080E090E0FC01EC54FB4F09C0E4EBAE
:101D8000F4E080E090E0019621912111FCCFF3CFA7
:101D9000CF01845B94408F3F910509F010F41192BC
:101DA000F7CF8091DD05865E60E071E002C0759539
:101DB00067958A95E2F70DC160E0C8010E94DE18C0
:101DC000882319F00F5F1F4FF7CF1093B5040093CE
:101DD000B40440E062E070E0FDC08091DE05815017
:101DE000843118F084E18093DE050091DE05809057
:101DF000FC059090FD05A090FE05B090FF0510E059
:101E00008FE2D82E60E080E090E00E94DE18E09142
:101E1000BE05F091BF05882309F450C08091B80534
:101E200084FF4CC08091B4048E3209F047C0809189
:101E3000B5048E3209F042C0011107C0A12FB0E0F5
:101E4000AC54BB4F8FE38C9339C001504480558014
:101E50006680778080819181A281B381848395831C
:101E6000A683B783E12CF12C60E0C7010E94DE1845
:101E7000882341F2E091BE05F091BF0580819181F8
:101E8000A281B381481659066A067B0699F41C5054
:101E9000E12FF0E0DF01AC54BB4FDC92A4EBB4E0E7
:101EA000EB54FB4FCF010B962D9121938E179F077B
:101EB000D9F7A8CFEFEFEE1AFE0AD6CF848295822B
:101EC000A682B782812F90E0DC01AC54BB4F119504
:101ED00020E03D91E22FF0E0EC54FB4F30832F5F88
:101EE0002113F7CF8195811103C01092B40481E0D2
:101EF000E82FF0E0EC54FB4F10828F5FC9F7609140
:101F0000DE05FCE06F9FB001112463C0153008F0BE
:101F100048CE28E1129FF0011124E45CFD4FF093BC
:101F2000BF05E093BE058091FC059091FD05A09151
:101F3000FE05B091FF0584839583A683B78331CED8
:101F40009C91891709F43BCE21C01530D0F488E16B
:101F5000189FF0011124E45CFD4FF093BF05E0935E
:101F6000BE058091FC059091FD05A091FE05B09104
:101F7000FF0584839583A683B78360E0C7010E9431
:101F8000DE18F092DF05E092DE05B7C09FEFE91A98
:101F9000F90A07CE8091DD05803F08F0D9C1BACD9E
:101FA0008091DE05853008F081E08093C0050E94B5
:101FB0004605BEC16091DE05E091DF05F0E0E0542A
:101FC000FA4FA4EBB4E0862F91919D938150E1F7F5
:101FD00070E040E084EB94E00E941220CAC160E00F
:101FE00080E090E00E94DE18811116C08091DE052D
:101FF000882309F49DC1E091BE05F091BF05809151
:10200000380290913902A0913A02B0913B02848348
:102010009583A683B7837ECD8091B80584FFE6CFF4
:102020008091B4048E3211F78091B5048E32F1F6AE
:10203000E091BE05F091BF05C480D580E680F780B1
:1020400080819181A281B38184839583A683B783A4
:102050008091DE05882351F200E010E060E0C801C5
:102060000E94DE18882311F2E091BE05F091BF05B1
:1020700080819181A281B381C816D906EA06FB0648
:1020800009F4A7CD0F5F1F4FE9CF809138029091DF
:102090003902A0913A02B0913B028093FC059093E3
:1020A000FD05A093FE05B093FF0560E080E090E0A1
:1020B0000E94DE183DC11530B0F4A8E11A9FF0016E
:1020C0001124E45CFD4FF093BF05E093BE058091C1
:1020D000FC059091FD05A091FE05B091FF0584835C
:1020E0009583A683B78360E08091DE059091DF053C
:1020F0000E94DE18882309F42BC19091B805E09165
:10210000BE05F091BF0594FF09C080819181A28135
:10211000B38184839583A683B78301C140815181B4
:102120006281738140875187628773871486158621
:102130001686178686898870868B90FD02C0178A5E
:1021400002C081E0878B8091BC04813409F049C0D2
:102150008091BD04843509F0B1C08091BE04823500
:1021600009F0A1C020E130E040E050E0BA0180E099
:102170000E94E61AE090BE05F090BF05F70186893F
:10218000982F9160968B2091B8049091B904922B6E
:10219000913011F48162868BF70182899389A48939
:1021A000B589BC01CD016051710981099109D688B9
:1021B000D5FE05C020E031E040E050E004C020E85A
:1021C00030E040E050E00E94C834213D32404105FB
:1021D000510508F47AC08D2D8068D70156968C93EE
:1021E00074C0883559F48091BD04863409F066C006
:1021F0008091BE04843409F061C01AC0833459F45C
:102200008091BD04813409F059C08091BE048335AA
:1022100009F054C00DC0823409F050C08091BD0453
:10222000893409F04BC08091BE048E3409F046C059
:1022300024E030E040E050E0BA0180E00E94E61A7D
:102240008091B404863469F48091B504853579F4BD
:102250008091B6048A3459F48091B704893439F4F2
:102260002DC08F3F21F48091B5048F3F39F1E0916B
:10227000BE05F091BF058689982F9161968B4289A2
:102280005389648975894130B8E65B07B1E06B0713
:102290007105D8F0413058406240710510F48169F1
:1022A00013C0816311C0883549F40E94BF2FE091AB
:1022B000BE05F091BF058689836006C0E091BE052A
:1022C000F091BF058689816C868B8FEF810F8430FA
:1022D00030F560E08091DE059091DF050E94DE1808
:1022E00084EB94E00E94E020E0914001F0914101F4
:1022F0000280F381E02D34E1139FE00DF11D1124E4
:10230000859194914CE050E064EB74E003960E9458
:10231000F23780912102811102C00E946423E09172
:10232000BE05F091BF05868983FF02C00C94990811
:1023300080910F02882321F083E40E94EC0506C0FF
:102340008FE79CE00197F1F700C0000083E40FC025
:1023500080910F02882321F085E40E94EC0506C0DD
:10236000AFE7BCE01197F1F700C0000085E40E94E0
:102370007A1F2796E2E10C945C35A4E0B0E0E3EC30
:10238000F1E10C944035459A3D9882E080936800D5
:1023900080E280936C0080B7846880BF8FE0809378
:1023A0007E0083B5816083BD84E79BEC90938900B8
:1023B0008093880080916F00826080936F001092FC
:1023C000C1051092C3051092C0051092B605109277
:1023D000BD0580E690E00E94E83D8093C2050E9422
:1023E0009E27E0914001F09141010190F081E02DA4
:1023F000099580913F0182FF03C081E08093C00571
:1024000088E690E00E94611F61E08091B6050E941D
:102410000C050E9479152FEF31EE44E02150304039
:102420004040E1F700C000000E94BF158823E1F1A1
:102430001F928F9385E891E09F938F9384EB94E0B4
:102440009F938F930E94013884EB94E00E94C826EA
:102450008091BB028F938091BA028F938091B902D1
:102460008F938091B8028F938091B7028F93809160
:10247000B6028F938091B5028F938091B4028F93AF
:1024800087E791E09F938F9324EB34E03F932F9362
:102490000E94013884EB94E00E94C8260FB6F8949D
:1024A000DEBF0FBECDBF7AC08DB581608DBD8CB54E
:1024B0008D7F8CBD8CB58E7F8CBD10925202109298
:1024C0006A021092820210929A021092B2020E9444
:1024D0008B178823B9F01F928F9384E691E09F9326
:1024E0008F9384EB94E09F938F930E94013884EB49
:1024F00094E00E94C8260F900F900F900F900F90BD
:102500000F904CC089E08093210266E9E62E61E0DD
:10251000F62E91E09B83C7010E94F03D6093FC057D
:102520007093FD058093FE059093FF056F3F7F4FED
:102530008F4F9F4F89F0C70104960E94F63D9093FC
:10254000DF058093DE058B81806F8093DD05F1E7E9
:10255000F093DC050E9491072B812F5F2B8336E0DF
:10256000E30EF11C2530B9F6109221020E9464237B
:102570008091380290913902A0913A02B0913B02C9
:102580008093FC059093FD05A093FE05B093FF0595
:102590000E9402078091C0050E94460560E080917C
:1025A000B6050E940C057894612C712C44EB54E024
:1025B0005C834B83212C312C210158E1852E0E9414
:1025C0003C2E882309F45AC18091700080FF03C01B
:1025D0000E9428063EC10E947328009709F446C154
:1025E00010922406FC017096259134913C832B8334
:1025F0003A832983FC01C590D4907601F89448EF82
:1026000055E05093BF054093BE0520912102211152
:1026100016C0F6012081243491F4E0914001F0913C
:10262000410122813381AC01421B530B9A01359544
:102630002795359527955DEC259F902C1124FC015D
:10264000729625913491F90109958C0178948091C5
:10265000C005981679F0EB81FC81808182FF0AC069
:102660009092C005911002C00E9402078091C0059F
:102670000E944605F60180818E33A9F4899CF00101
:102680001124E45CFD4F008911890F5F1F4F848185
:102690009581A681B781E091BE05F091BF05848345
:1026A0009583A683B78301151105F9F0F8940F3FC0
:1026B000FFEF1F0731F422EE2093DD059092DE0537
:1026C0000EC0899CF0011124E45CFD4F168A892D0F
:1026D000806F8093DD051093DF050093DE0531E701
:1026E0003093DC050E94910778948091210281113A
:1026F00028C0F60180818E3421F58091C0058823A1
:1027000001F1889EF0011124E45CFD4F96899860E8
:10271000968BE0914001F09141010280F381E02D20
:1027200024E1829FE00DF11D1124E590F4904CE02E
:1027300050E067E571E0C70103960E94E3370E940D
:10274000642380912102833009F073C0F7018081F6
:10275000833509F073C0E0914001F0914101018897
:10276000F289E02DB496A591B4918091B70580FDD2
:1027700003C08C9182FF21C08091B7058E7F80932A
:10278000B705EB81FC8180818B7F80838C918B7F6F
:102790008C9329E4E22E21E0F22E0AE812E520EEE5
:1027A0003FEF42E064E870E083E290E00E94702C2A
:1027B0000E946423612C712C41C0E091BE05F09110
:1027C000BF0580819181A281B38180879187A28793
:1027D000B3870E943C338091B70581608093B70531
:1027E000EB81FC8180818460808399E3E92E91E014
:1027F000F92E0AE812E520EE3FEF42E064E870E0CF
:1028000083E290E00E94702C0E9464238091B705BF
:1028100081FD19C0FAEA26EE36E941E0F150204088
:1028200030404040D9F7000084EB94E09C838B83D8
:102830000EC0E4EBF4E0FC83EB8309C024EB34E04E
:102840003C832B8304C044EB54E05C834B8300E265
:102850001EE40E943C2E8111FCCF5FEF80E792E0E6
:10286000515080409040E1F700C0000010920902F2
:1028700010920A0210920B0210920C028091B7057E
:1028800080FF24C0F8948091B70581FF04C0C30184
:102890000E946F3303C0C3010E9484323C01892B24
:1028A00021F08091B70580FD10C088E690E00E947D
:1028B000611F8091B7058E7F8093B705E981FA810A
:1028C00080818B7F80830E946423789480913F0174
:1028D00081FF5AC080912102813009F055C0F090EB
:1028E0002406FF2009F450C00032FEE41F0709F05F
:1028F00049C023E12F1518F01092240602C083E18D
:10290000F82E40913B0150913C0141505109A12CBE
:10291000B12CC12CD12CE12C01E02AE130E06AE09D
:1029200070E085E090E00E94CB2ACF2CEB80FC8009
:1029300000E010E020EE3FEF42E06AE070E085E06A
:1029400090E00E94B82C4B815C8184E0443B5807A6
:1029500069F0FA0101900020E9F7CF01449784174C
:10296000950739F4E3EBF4E0FC83EB8302E21EE429
:1029700002C000E010E02B813C812F5F3F4F3C8381
:102980002B8302C00E5F1F4F31EA231630EF330650
:1029900039E14306510430F00E941E17212C312CDE
:1029A000210105C04FEF241A340A440A540A8091C9
:1029B0003F0184FF04CE80912102811100CE8091DD
:1029C000090290910A02A0910B02B0910C02813889
:1029D00054E895075EE1A507B10538F080917000D5
:1029E0008111EDCD0E941906EACD0196A11DB11D00
:1029F0008093090290930A02A0930B02B0930C02F9
:102A0000DECD1F920F920FB60F9211242F933F939A
:102A10004F935F936F937F938F939F93AF93BF93E6
:102A2000EF93FF93359929C08091000190910101A6
:102A30009093BF058093BE05109224061092DD0589
:102A40000E94910760E08091B6050E940C0580917C
:102A5000BE059091BF05909301018093000188EF1E
:102A600095E09093BF058093BE05109209021092E5
:102A70000A0210920B0210920C02FF91EF91BF918B
:102A8000AF919F918F917F916F915F914F913F9106
:102A90002F910F900FBE0F901F9018952A9A229A8F
:102AA0002D9A259A2498239A8DB58E7F8DBD83E526
:102AB0008CBD8DB508958EBD0DB407FEFDCF8EB5CE
:102AC00008958FEF0E945B150895FB01E40FF51F39
:102AD00039E06E177F0761F0229198E0880F482F48
:102AE000422747FD8327220F9150C1F78F77F1CFFF
:102AF00008950E944E150895A5E0B0E0E2E8F5E1E2
:102B00000C944F354A835B836C837D838064898317
:102B10000E945B158D810E945B158C810E945B1564
:102B20008B810E945B158A810E945B1541E050E019
:102B3000BE016F5F7F4F80E00E94651544E050E06A
:102B4000BE016E5F7F4F0E946515880F81600E94F5
:102B50005B151FEF0E946115115011F087FDFACF30
:102B60002596E3E00C946B35CF932A980E947C1550
:102B7000C82F2A9A0E9461158C2FCF910895EF9249
:102B8000FF920F931F93CF93DF938FEF9FEFDC01A3
:102B90008093110690931206A0931306B093140627
:102BA00010921506809110068E7F80931006CAE061
:102BB0000E946115C150E1F7DAE040E050E0BA014F
:102BC00080E00E94B415813031F0D150B1F780938C
:102BD000B402C1E091C084EBE82E82E0F82E1AE046
:102BE0002A984AEA51E060E070E088E00E947C1593
:102BF000D82F8130C1F4870184E0E80EF11C0E94D7
:102C00006115F80181938F01EE16FF06C1F78091DF
:102C1000B602813031F48091B70210E08A3A11F4A3
:102C200002C010E0D6E02A9A0E9461158D2F8B7F9A
:102C3000813061F08FEF810F112311F0182FD0CF69
:102C4000D63020F0F701D083C2E056C00FEF13E07A
:102C500040E050E0BA0187E30E94B415D82F8230DB
:102C6000A8F540E050E060E070E489E20E94B4150D
:102C7000811127C02A9840E050E0BA018AE30E94FF
:102C80007C15D82F0E9461158093B8020E946115AF
:102C90008093B9020E9461158093BA020E94611567
:102CA0008093BB022A9A0E9461158091B80286FB2C
:102CB000882780F99091100680FB90F99093100678
:102CC00005C00150110921F6C3E016C0D53041F40A
:102CD00040E050E0BA0181E00E94B41581110BC0C0
:102CE00040E052E060E070E080E10E94B41588238B
:102CF00019F0C5E001C0C4E08C2FCDB7DEB7E6E027
:102D00000C946835CF93DF93AB01BC012A98809176
:102D1000100680FD07C089E0440F551F661F771F0E
:102D20008A95D1F781E10E947C15811115C00E941E
:102D300061158E3FE1F7C4EBD2E00E9461158993E3
:102D400084E0C43BD807C9F70E9461150E94611551
:102D50002A9A0E94611580E0DF91CF910895CF9368
:102D6000DF93AB01BC012A988091100680FD07C05B
:102D700089E0440F551F661F771F8A95D1F788E1B8
:102D80000E947C15811120C00E9461158EEF0E9467
:102D90005B15C4EBD2E089910E945B1584E0C43BD3
:102DA000D807C9F70E9461150E9461150E9461153C
:102DB000982F9F71953041F40E9461158823E1F3AB
:102DC0002A9A0E94611580E0DF91CF9108950F93B8
:102DD0001F93CF93C82F00E018EF21E043E050E0AD
:102DE00065E070E08FE090E00E94202BCC23F1F0B2
:102DF000C0E16091110670911206809113069091C6
:102E000014060E94AF16882319F0C15091F7FFCF26
:102E10001092150600E010E021E043E050E065E08C
:102E200070E08FE090E00E94202B03C081E080934F
:102E3000150680E0CF911F910F910895809115069E
:102E4000882321F081E00E94E716FACF0895CF92FF
:102E5000DF92EF92FF92CF93C0901106D0901206AE
:102E6000E0901306F0901406C616D706E806F90699
:102E700011F48FEF18C06B017C010E941E17C0E097
:102E8000C701B6010E948216C150882319F0C111F2
:102E9000F7CFEFCFC0921106D0921206E092130640
:102EA000F092140680E0CF91FF90EF90DF90CF90EA
:102EB0000895CF92DF92EF92FF92C0902F02D090B0
:102EC0003002E0903102F090320261157105810507
:102ED000910569F48091330290913402A701960123
:102EE000281B390B41095109CA01B9010FC09B01C7
:102EF000AC012250310941095109A0913702B0E0DB
:102F00000E942D356C0D7D1D8E1D9F1DFF90EF9035
:102F1000DF90CF900895A0E0B0E0E1E9F7E10C94F4
:102F2000423560E070E0CB010E9427178111E8C0B4
:102F3000D091760480907A0490907B04A0907C04D9
:102F4000B0907D04C501B4010E942717C82F8111DC
:102F5000D9C0E091C502F091C60284E0F695E795EC
:102F60008A95E1F7F0933402E09333028091CA022C
:102F70009091CB02009719F0A0E0B0E008C08091DA
:102F8000D8029091D902A091DA02B091DB0280932D
:102F90002B0290932C02A0932D02B0932E02C0908E
:102FA000C202D090C302E12CF12CA091C402209166
:102FB0002B0230912C0240912D0250912E02B0E054
:102FC0000E942D352B013C01B501A4014C0D5D1D66
:102FD0006E1D7F1D8F0120E030E0D301C201840F00
:102FE000951FA61FB71F800F911FA21FB31F8093AD
:102FF0002F0290933002A0933102B093320280915D
:10300000C7029091C802009719F0A0E0B0E008C094
:103010008091D4029091D502A091D602B091D702AE
:1030200084199509A609B7098C199D09AE09BF092C
:10303000801B910BA20BB30B80932302909324026D
:10304000A0932502B09326028091C102809337029B
:103050008091BF029091C002909336028093350216
:1030600040932702509328026093290270932A020A
:103070008FEF9FEFDC018093160690931706A093C5
:103080001806B0931906DD3038F4DB3098F4D430EC
:1030900029F0D630C9F502C0DE30B1F5E091BE05A9
:1030A000F091BF0514821582168217828091100656
:1030B0008D7F13C08091E0029091E102A091E20225
:1030C000B091E302E091BE05F091BF058483958342
:1030D000A683B78380911006826080931006E091EA
:1030E000BE05F091BF0584819581A681B78180934B
:1030F000380290933902A0933A02B0933B0205C084
:10310000C1E003C0C2E001C0C3E08C2FCDB7DEB781
:10311000E0E10C945E358F929F92AF92BF92CF9276
:10312000DF92EF92FF922091100621FF0EC042E045
:10313000660F771F881F991F4A95D1F7CC24CA9430
:10314000DC2CEC2C5FE0F52E09C0660F771F881F82
:10315000991FCC24CA94DC2CE12CF12C209135024F
:103160003091360240E050E00E94C8344B015C01CF
:103170008091270290912802A0912902B0912A0201
:10318000BC01CD01620F731F841F951F0E9427177A
:10319000F401EC54FD4F80819181A281B381BC0187
:1031A000CD016C217D218E219F21FF90EF90DF903A
:1031B000CF90BF90AF909F908F900895AAE0B0E01D
:1031C000E4EEF8E10C9440351C016A83E091BE0501
:1031D000F091BF05C480D580E680F7808091160607
:1031E00090911706A0911806B0911906C816D90635
:1031F000EA06FB0651F0C0921606D0921706E0923E
:103200001806F092190610921A0680911A06882361
:1032100089F020911A0230911B023E832D832215E2
:10322000330598F02215330529F4813019F43A81D9
:10323000332359F0C701B6010E9459172B013C01F5
:1032400010E01E821D82198240C000911002809001
:10325000160290901702A0901802B0901902C09028
:103260001102D0901202E0901302F090140210911B
:1032700015021982240135018FEF481A580A680A8D
:10328000780AC501B4010E94271790E2099FF00156
:103290001124EC54FD4F4081442309F4E9C0453E1C
:1032A000C9F4B0960F5F0031B1F7C114D104E10445
:1032B000F10409F0CCC0812F90E0209133023091CD
:1032C00034028217930708F0BBC01F5F530142010D
:1032D00000E0D0CF83858F3009F053C0AA81AA23A4
:1032E00001F3842F90E001978F709927BDE0B89F7C
:1032F000B001B99F700D11246C547B4F9F017A87E8
:103300006987CF010A969C838B83F887EF83AF810F
:10331000B88511965C91A985BA855D93BA87A9870E
:103320008F819885029698878F83AB81BC818A179D
:103330009B0769F7CB0105969C838B83CF010C9685
:10334000D9011E965C91AB81BC815D93BC83AB833C
:103350002E5F3F4F8217930799F7848DDB011B96F1
:103360008C931B97868D1C968C931C9746FF02C0EE
:103370001D961C924F70413009F093CF31E0398394
:1033800090CFB981BB2361F02D813E812215330599
:1033900009F470C02F5F3F4F3E832D83198281CF88
:1033A0004E3229F49181903211F484FD7ACF83FD5D
:1033B00078CF8D819E8182159305D9F5CF0164EB7D
:1033C00074E0AB01DC012D91CD01DA012D93AD014B
:1033D000B4E04F3B5B07B1F71092BF042A81222370
:1033E00009F44AC01092C0048091BE048093BF04C7
:1033F0008091BD048093BE048091BC048093BD0481
:103400008091B4048E3219F08EE28093BC0424EBD8
:1034100034E0DB018D91BD01803221F0D9018C9324
:103420002F5F3F4FDB018C918111F3CFD9011C92AB
:1034300023C02D813E812F5F3F4F3E832D8331CFAF
:1034400090911006892F827091FD3FCF6EC08091C0
:103450003702181708F439CFC701B6010E948B183C
:103460006B017C010E9459172B013C0110E02DCF0C
:1034700080E005C082E003C03E822D8281E0A09101
:10348000BE05B091BF054489558960E070E0BA017E
:1034900055274427228D338D2901612C712C442915
:1034A0005529662977294D935D936D937C931397E6
:1034B00051963C922E925097448D558D668D778D06
:1034C00052964D935D936D937C935597938590930E
:1034D000B805268937893093BC052093BB05208D1C
:1034E000318D3093BA052093B9058823E9F0AD8179
:1034F000BE81B0931B02A0931A0200931002809227
:10350000160290921702A0921802B0921902C0926D
:103510001102D0921202E0921302F0921402109360
:10352000150280931A0601C080E02A96E2E10C940D
:103530005C35A0E0B0E0EFE9FAE10C944A356B01AC
:103540007C01E091BE05F091BF0584859585A68537
:10355000B785C816D906EA06FB0660F4808191811A
:10356000A281B38180879187A287B387148615864D
:1035700016861786C091BE05D091BF050C851D85A6
:103580002E853F85688579858A859B85C016D106FD
:10359000E206F306B1F00E948B18688779878A8764
:1035A0009B87E091BE05F091BF0584859585A68532
:1035B000B7850196A11DB11D84879587A687B7871A
:1035C000D9CFCDB7DEB7E8E00C946635A9E0B0E01E
:1035D000ECEEFAE10C944035E091BE05F091BF05A8
:1035E00042885388648875884415550566057705B3
:1035F00018F080E090E0E2C019016A017B018D8340
:1036000020913702A0913502B0913602AD0160E001
:1036100070E04E835F836887798730E00E941735BA
:103620004B015C01C301B2016C197D098E099F0930
:1036300069837A838B839C83C701B601A5019401BA
:103640000E94C83429013A01A5019401C301B201C5
:103650000E948434C61AD70AE80AF90AC701B601DB
:103660002E813F81488559850E94C83449015A01FD
:103670002E813F8148855985C501B4010E9484345B
:10368000C61AD70AE80AF90AC301B2010E94991AB8
:10369000E091BE05F091BF056085718582859385B7
:1036A0000E945917680D791D8A1D9B1D0E942717BE
:1036B00004EB14E01F821E828E819F818215930588
:1036C00009F44BC08091350290913602A0E0B0E041
:1036D000C816D906EA06FB06C0F17D817130E1F01B
:1036E0008FEF881A980AA80AB80A8091370290E0EA
:1036F000A0E0B0E088169906AA06BB0698F09FEFF6
:10370000491A590A690A790AC301B2010E94991A31
:10371000812C912C540106C080E00E94E71688237A
:10372000F9F267CFE091BE05F091BF056085718524
:10373000828593850E945917680D791D8A1D9B1DEE
:103740000E942717C12CD12C760149815A816B81A7
:103750007C81452B462B472B21F45D81513061F54F
:1037600026C0F601EC54FD4F6D81613019F4D8018B
:103770008C9102C08081F801808349815A816B81DC
:103780007C81415051096109710949835A836B83D6
:103790007C836E817F816F5F7F4F7F836E837FEF3E
:1037A000C71AD70AE70AF70A0F5F1F4F85CF80E0D5
:1037B0000E94E71681111DCF8E819F812996E2E13B
:1037C0000C945C35AAE1B0E0E8EEFBE10C944035E6
:1037D0009C878B87788F6F8BDC018D909D90AD904F
:1037E000BC90BFEF8B1A9B0AAB0ABB0A80911006F4
:1037F000209035023090360281FF11C03694279414
:10380000369427942FEF3FEF4FEF5FE02F833887F9
:1038100049875A8744E050E05E834D830EC036945A
:1038200027948FEF9FEFA0E0B0E08F839887A98760
:10383000BA87A2E0B0E0BE83AD836101E12CF12C38
:10384000C501B401A70196010E94C83429013A01BB
:10385000A7019601C301B2010E94843469837A836F
:103860008B839C838091270290912802A09129024A
:10387000B0912A02480E591E6A1E7B1E40912702F3
:10388000509128026091290270912A0280912B02A6
:1038900090912C02A0912D02B0912E02840F951FC1
:1038A000A61FB71F481659066A067B0608F0C4C053
:1038B000C301B2010E942717C501B401A7019601F7
:1038C0000E94C8347A8F698F8090270290902802D6
:1038D000A0902902B0902A0200912B0210912C0294
:1038E00020912D0230912E02800E911EA21EB31E39
:1038F000A501940121503109410951092D873E87C5
:103900004F87588B20912302309124024091250249
:1039100050912602298B3A8B4B8B5C8B809037021F
:10392000912CA12CB12CAD81BE81A69FA001A79F97
:10393000500DB69F500D11245E8B4D8B00E010E0B2
:10394000498D5A8D4215530508F061C02D853E857D
:103950004F8558894216530664067506E9F469894D
:103960007A898B899C89A50194010E94C834CA0177
:10397000B901A70196010E94C834DC01CB01019670
:10398000A11DB11DE98DFA8DAF0160E070E08417D3
:103990009507A607B707D8F1ED89FE89E00FF11F5B
:1039A000EC54FD4F80819181A281B3812F813885B4
:1039B00049855A8582239323A423B5234D815E81B3
:1039C000040F151F892B8A2B8B2BD1F4C980DA8029
:1039D000EB80FC80898D9A8DC80ED91EE11CF11CEC
:1039E000AB85BC85CD92DD92ED92FC921397EF8969
:1039F000F88D408251826282738280E090E01EC026
:103A0000298D3A8D2F5F3F4F3A8F298F99CF89812A
:103A10009A81AB81BC818C0D9D1DAE1DBF1D89831C
:103A20009A83AB83BC839FEF491A590A690A790AC2
:103A3000812C912C540122CF81E090E06A96E2E142
:103A40000C945C35A9E1B0E0E8E2FDE10C9440356E
:103A50005C016A017B0120911602309117024091AE
:103A60001802509119022E873F87488B598B00917D
:103A7000100210E00F5F1F4F0F7011270115110585
:103A800041F42F5F3F4F4F4F5F4F2E873F87488B4B
:103A9000598B8091100681FD0DC08FEF9FEFA0E044
:103AA000B0E08A8B9B8BAC8BBD8BA2E0B0E0BD8776
:103AB000AC870CC02FEF3FEF4FEF5FE02A8B3B8BC3
:103AC0004C8B5D8B44E050E05D874C8719821A82F5
:103AD0001B821C82BE016B5F7F4FCE0101960E944C
:103AE000E21B892B29F060E070E080E090E046C1A5
:103AF0006E857F85888999890E94271785E0000F48
:103B0000111F8A95E1F7C8018C549D4F9A878987C8
:103B100089819A81AB81BC81E985FA85B58BA48BBB
:103B2000938F828F48E050E0B501CF010E94F237B9
:103B300043E050E06AE272E089859A8508960E9427
:103B4000E337A985BA855C96CD92DD92ED92FC9221
:103B50005F9780E21B968C9380E00E94E7168111AC
:103B6000C2CF89809A80AB80BC80C501B4010E941D
:103B700059176E8B7F8B888F998F209035023090EC
:103B80003602B0913702BB87910140E050E0C70197
:103B9000B6010E94C834EB854E2E512C612C712C3D
:103BA000CA01B901A30192010E94C8348901FB85B1
:103BB000F29D9001F39D300D112440E050E0C701CB
:103BC000B6010E94C834672B682B692B11F4015091
:103BD0001109C1016C857D850E94A0349B0140E0E4
:103BE00050E0C501B4010E94C83480912702909131
:103BF0002802A0912902B0912A02820F931FA41FCC
:103C0000B51F8D839E83AF83B887612C712C1B8673
:103C10002C853D851901412C512C809135029091C4
:103C200036026C857D850E94A0349B0140E050E007
:103C300069817A818B819C810E94C8349B01AC018F
:103C4000C201B1010E9484346B017C018D809E8091
:103C5000AF80B884BE016B5F7F4FCE0101960E949A
:103C6000E21B892B21F03B853F5F3B8783018D81E0
:103C70009E81AF81B88588169906AA06BB0621F0F9
:103C8000C501B4010E94271780911006F601EC547B
:103C9000FD4F60167106A0F481FF0DC089819A81E5
:103CA000AB81BC812A893B894C895D89822393231E
:103CB000A423B5230BC089819A81918380830FC08F
:103CC00081FF09C08A899B89AC89BD8980839183E2
:103CD000A283B38304C0AFEFBFEFB183A08380E0C2
:103CE0000E94E71680912B0290912C02A0912D0248
:103CF000B0912E02BC01CD01680D791D8A1D9B1D5E
:103D00000E94AF16BFEF6B1A7B0A0615170508F065
:103D100084CFEB85EE2331F16E857F858889998983
:103D20000E94271720913702809135029091360228
:103D3000289FA001299F500D1124C8010196489F7A
:103D40009001499F300D589F300D1124C901A0E00A
:103D5000B0E0E985FA85848F958FA68FB78F81E0D3
:103D60000E94E71680911A0290911B0260E0019672
:103D70000E94DE186E897F89888D998D6996E2E1AF
:103D80000C945C35ABE0B0E0E8ECFEE10C9442351D
:103D90001B861A86611571058105910521F460E085
:103DA00070E0CB017BC04091370220913502309109
:103DB0003602429FF001439FF00D11248F0120E055
:103DC00030E0980111270027061717072807390741
:103DD00030F32B013C01E091BE05F091BF058091CD
:103DE000160690911706A0911806B09119068483C3
:103DF0009583A683B78380E090E000E010E04E0159
:103E00002AE0820E911C22E2C22E22E0D22E34EB56
:103E1000A32E34E0B32E7C012FEFE21AF20A60E009
:103E20000E94DE188823B1F09F928F92DF92CF928A
:103E3000BF92AF920E9423388A859B850F900F9086
:103E40000F900F900F900F900817190708F48C012E
:103E5000C701E1CF81E0E816F10409F4A0CF0F5FBC
:103E60001F4F003127E2120708F099CF1F930F93DD
:103E700089E192E09F938F938E010F5F1F4F1F93F5
:103E80000F930E940138B301A201C8010E94221DB4
:103E90000F900F900F900F900F900F902B96E0E1E6
:103EA0000C945E35FC01680F791F80E0E617F70778
:103EB00039F09191980F981708F49F5F892FF6CFEA
:103EC00008952091C00025FFFCCF9093C5008093FA
:103ED000C40082E28093C00088E18093C10087E043
:103EE0008093C2008091C00087FF03C08091C6000C
:103EF000F9CF08959091C00095FFFCCF8093C60044
:103F000008950F931F93CF93DF93EC018C01060F5D
:103F1000171FC017D10721F089910E947A1FF9CF8E
:103F2000DF91CF911F910F910895CF92DF92EF9281
:103F3000FF92CF93DF939B01FC0152EFC52E59E412
:103F4000D52E52E0E52EF12C50E0A6B1A072B0E0E3
:103F5000A417B50711F5A1E0CA1AD108E108F108C4
:103F6000F1F0A091C000A7FFF0CFA091C000D091C8
:103F7000C600A4FD16C0CA2FC870A3FD14C0211529
:103F8000310531F40E94521FD81771F0C0E80CC0FF
:103F9000D083215031093196D8CFC1E005C0C2E0AD
:103FA00003C0C3E001C0C4E08C2FDF91CF91FF902C
:103FB000EF90DF90CF900895A1E0B0E0E2EEFFE156
:103FC0000C94503540E20E94951F89838FE99FE051
:103FD0000197F1F700C000008981882391F08EE4F9
:103FE0000E947A1F80910F028823B9F08EE40E940C
:103FF000EC058981805D8983CE0101960E94C826E7
:104000000CC081E40E947A1F80910F02882331F056
:1040100081E40E94EC0580E001C08FEF2196E2E090
:104020000C946C350F931F93CF93DF93EC018B01AE
:1040300080910F02882351F0442321F085E40E94EF
:10404000EC050CC083E40E94EC050AC08FE79CE0FD
:104050000197F1F700C00000442311F085E401C08E
:1040600083E40E947A1F8FE193E00197F1F700C08B
:104070000000B801CE010E94811FB801CE010E944C
:10408000521F0E947A1FDF91CF911F910F910895C7
:104090004096FC01A591B4918C9184608C9380E052
:1040A00090E0089581E0809321028093200278942B
:1040B000E0914001F09141010580F681E02D0995E4
:1040C00080E090E0089580912102813051F4809148
:1040D0001E0290911F020A9790931F0280931E0266
:1040E00004C010920F021092200210922102E0915F
:1040F0004001F09141010190F081E02D099580E0AF
:1041000090E008951092210280911E0290911F026A
:104110000A9790931F0280931E02809120028823A9
:1041200039F083E0809321021092500110924F01E8
:1041300080912102E0914001F091410195E0899F39
:10414000E00DF11D11240190F081E02D0995809181
:104150004F0190915001089582E080932102E091F7
:104160004001F09141010284F385E02D099580E042
:1041700090E0089580E090E00895FC0180911B0696
:1041800090911C06893C910568F081E080932102A2
:104190007894E0914001F09141010580F681E02D95
:1041A000099508C0889748F07096A591B4918C91B4
:1041B00084608C9380E090E008958FEF9FEF0895E6
:1041C000FC018285838781858287808581878EE255
:1041D000808714860895EF92FF920F931F93CF93D9
:1041E000DF9380911C0290911D02892B09F45AC023
:1041F00060E080911E0290911F020E94DE188823C9
:1042000009F4C6C060E270E08FE090E00E94DC2C10
:1042100020911C0230911D0282E491E09F938F93C4
:10422000C9010197EAE0F0E0BF010E94A0346F5F8E
:104230007F4F7F936F9380911E0290911F02BF0169
:104240000E94A0346F5F7F4F7F936F933F932F93B4
:1042500081E792E09F938F9384EB94E09F938F93F9
:104260000E94013824EB34E040E050E06FEF7FEF34
:1042700081E00E940D2D6DE270E08FE090E00E94E1
:10428000DC2CC0911E02D0911F028DB79EB70C96F8
:104290000FB6F8949EBF0FBE8DBF8FE0E82E85E06D
:1042A000F82E44C060E080911C0290911D020E9493
:1042B000DE18882309F49CCF80911C0290911D0286
:1042C000019690931D0280931C02ECCF60E0CE011A
:1042D0000E94DE18882309F44DC08091B805209112
:1042E000BC0484FD3AC08EEE94E0FC0134912317A7
:1042F00031F10396E816F906C1F70DE71FEE2032FB
:1043000091F184EB94E00E94E02080914F01909124
:10431000500124EB34E04AE852E5C817D90741F5CB
:1043200060EF7FEF82E00E940D2D219680911E02AA
:1043300090911F020A96C817D90740F225C03196FE
:10434000E4913091BD043E13D4CFFC013296E49148
:104350003091BE043E13CDCF03C00FEF17E0CFCF97
:1043600000EE17E0CCCF2093BF041092C004CDCF55
:10437000B801D8CF24E632E04AE852E560EE77E0B3
:1043800082E00E94E52CD1CFD0931F02C0931E0281
:1043900080E090E0CDB7DEB7E6E00C946835809120
:1043A0001E0290911F028431910538F0449790933A
:1043B0001F0280931E020E94EB2080E090E008958F
:1043C00010921F0210921E020E94EB2080E090E0EB
:1043D000089580911C0290911D0201976AE070E09F
:1043E0000E94A0342AE0269FC001279F900D11242F
:1043F00090931F0280931E020E94EB2080E090E0C9
:104400000895A5E0B0E0E7E0F2E20C94403580E0EA
:1044100090E00E94FA29198204E110E024E130E0E2
:104420003D832C838C809D803AE0830E911CAC8070
:10443000BD808AE0A81AB1082FEF3FEFA801B401B0
:10444000C5010E94BF2A68019AE0C90ED11C7801FB
:104450002AE0E21AF1082FEF3FEFA601B7018C81A5
:104460009D810E94B52A0E943C2E8111FCCF0E94A2
:104470003C2E8823E1F30E94A82F60931B067093C3
:104480001C0680931D0690931E0620EE37E0A801BF
:10449000B401C5010E94BF2A20EE37E0A601B70192
:1044A0008C819D810E94B52A60911B0670911C062B
:1044B00080911D0690911E0639813230D1F0333043
:1044C00019F1313051F03B011C0180913B01909179
:1044D0003C0144979D838C8324C02B01280E391EF8
:1044E0003694279400913D0110913E010451110929
:1044F00018C0460E571E569447949B838A8324E126
:1045000030E03D832C830DC0660E771E7694679451
:104510002A813B81820F931F9C01369527953B830F
:104520002A833FEF89E698E1315080409040E1F7DF
:1045300000C0000029812F5F2983243009F072CF49
:104540000E943C2E8111FCCF60913B0170913C0197
:1045500080E090E00E948C366B017C01C2018619DC
:1045600097099D838C83BC01990F880B990B0E943E
:104570008E364B015C0120E030E040E252E4C7019E
:10458000B6010E9477359B01AC01C501B4010E94C0
:10459000E435A70196010E941A370E9456362C81F5
:1045A0003D81621B730B77FF02C06F5F7F4F759574
:1045B0006795661A770A460E571E60913D01709105
:1045C0003E0180E090E00E948C366B017C018A8184
:1045D0009B81821993099D838C83BC01990F880B61
:1045E000990B0E948E364B015C0120E030E040E2E6
:1045F00052E4C701B6010E9477359B01AC01C501A9
:10460000B4010E94E435A70196010E941A370E9466
:1046100056362C813D81621B730B77FF02C06F5FA2
:104620007F4F75956795261A370A8A819B81860F79
:10463000971F9B838A839F938F933F922F925F92C2
:104640004F927F926F9285E492E09F938F9384EBD9
:1046500094E09F938F930E94013860913D01709187
:104660003E017695679524EBE22E24E0F22E00E0E1
:1046700010E02FEF3FEF41E084E190E00E94952CA5
:104680000FB6F894DEBF0FBECDBF0E943C2E88232C
:10469000E1F3B3018DEB91E00E941A3EB20189EB88
:1046A00091E00E941A3EB1018BEB91E00E941A3E0C
:1046B0006A817B8187EB91E00E941A3E80E090E066
:1046C0002596E2E10C945C35A7E1B0E0EAE6F3E27E
:1046D0000C9440351D8A80912102E0914001F091B7
:1046E000410195E0899FE00DF11D112484819D8990
:1046F000981708F082C0228133819D8984E1989FB8
:10470000A0011124DE01119680E090E0FA01E80F8B
:10471000F91FE20FF31FE491ED93019684319105A7
:10472000A9F7E989FA89E080E1FE63C0E2FE08C0EA
:10473000EFE1F0E0FC87EB8780EE9FEF988B8F87AF
:104740004B845C848D809E80E985FA85FF8BEE8B9F
:104750006B807C802F803884260C371CAD84BE840F
:10476000E0FAEE24E0F89F01280D391D620101E016
:10477000A101B401C3010E94CB2AC980DA802F8530
:104780003889C40106976E897F8976956795680F89
:10479000791F7601820142E0C3010A960E94952C9E
:1047A000F6018081843429F58181803311F124015F
:1047B000F8E14F0E511C310182E0681A710898E04F
:1047C000890E911CE2E12E1A310805E115E09201F3
:1047D000A301B401C1010E94352DF60183818C3300
:1047E00041F400E018EF9201A301B401C1010E945D
:1047F000642AFD89FF5FFD8B6ECF6796E2E10C9422
:104800005C354096FC01A591B4918C9182FB99276F
:1048100090F9909590FB82F98C938091B70582FB7B
:10482000992790F9909590FB82F98093B7050E94A3
:10483000642380E090E008954096FC01A591B49136
:104840008C9182FF08C08091B70581608093B70585
:104850008C918B7F09C08091B70580FF08C08E7F47
:104860008093B7058C9184608C930E94642380E0D0
:1048700090E008954096FC01A591B4918C9182FB43
:10488000992790F9909590FB82F98C930E9464236C
:1048900080E090E00895AF92BF92CF92DF92EF92C6
:1048A0000F93CF93DF93CBE3D1E0488159814B50F5
:1048B0005109A12CB12C8AE8C82E82E5D82EE12C12
:1048C00001E028E131E068E270E08AE090E00E94D7
:1048D000CB2A488159814B50510999E5C92E9EEC4C
:1048E000D92E00E028E131E068E270E08AE090E053
:1048F0000E94CB2A488159814C50510927E131E06F
:1049000069E270E08BE090E00E94CB2A0E94642371
:104910008FEF9FEF9093500180934F010E94EB2007
:10492000DF91CF910F91EF90DF90CF90BF90AF903C
:104930000895AF92BF92CF92DF92EF920F93CF93F1
:1049400040913B0150913C014B505109A12CB12C9D
:104950008AE8C82E82E5D82EE12C01E028E131E07A
:1049600068E270E08AE090E00E94CB2A40913B012F
:1049700050913C014B50510999E5C92E9EECD92E1E
:1049800000E028E131E068E270E08AE090E00E9417
:10499000CB2A40913B0150913C014C50510927E1F9
:1049A00031E069E270E08BE090E00E94CB2A6091F8
:1049B00040017091410140E050E020E030E0809102
:1049C0002102FB0195E0899FE00DF11D11248481F6
:1049D00090E002972817390750F50280F381E02D07
:1049E000E40FF51F7096A591B491E0913F01F0E0BE
:1049F000022E02C0F595E7950A94E2F78C91E0FB50
:104A000082F98C9390912102FB01C5E09C9FE00DFF
:104A1000F11D1124E481F0E033972E173F0711F4C4
:104A20008B7F8C932F5F3F4F4C5E5F4FC8CF0E94B0
:104A30006423CF910F91EF90DF90CF90BF90AF9014
:104A40000895A0E0B0E0E7E2F5E20C944835CBE34E
:104A5000D1E04881598146505109A12CB12C8AE8F6
:104A6000C82E82E5D82EE12C01E025EF30E064E687
:104A700070E085E090E00E94CB2A48815981465041
:104A8000510999E5C92E9EECD92E00E025EF30E0C2
:104A900064E670E085E090E00E94CB2A488159816D
:104AA0004750510924EF30E065E670E086E090E081
:104AB0000E94CB2A2CE3E22E22E0F22E0AE812E535
:104AC00028E03CEF42E069E670E086E490E00E9476
:104AD000702C688179816850710928E03CEF4AE7C1
:104AE00050E087E090E00E94BF2A0E946423CDB787
:104AF000DEB7EAE00C946435A0E0B0E0E2E8F5E26D
:104B00000C944835EC01162F60911F067091200619
:104B100080913D0190913E0140978617970718F4C8
:104B200081E0809323069B01295F3F4F40913B0129
:104B300050913C014B505109A12CB12C8BE7C82E50
:104B400085E2D82EE12C01E0809121069091220689
:104B50000E94CB2A60911F06709120068091210649
:104B6000909122067E01112341F00BE715E22FEF11
:104B70003FEF41E00E94702C07C00BE715E22FEFDA
:104B80003FEF41E00E94952C80911F0690912006F6
:104B900008969093200680931F06209123062223D7
:104BA000E1F020913D0130913E0128503109281754
:104BB000390768F480912102843019F48AE090E08A
:104BC00002C08CE191E09093200680931F068091B3
:104BD0001F06909120060E94F929CDB7DEB7EAE0C2
:104BE0000C94643561E00E947C250895A0E0B0E05B
:104BF000ECEFF5E20C94483584E190E090932206C6
:104C0000809321068CE191E09093200680931F060B
:104C10000E94732944E050E060E270E080911F063A
:104C2000909120060E94F82980911F0690912006FD
:104C30000E94F9290E946B2980E090E00E94FA29E5
:104C40008EE0E82E82E0F82E00E010E028E03CEF55
:104C500042E06AE070E084E190E00E94702C92E013
:104C6000E92E92E0F92E28E03CEF41E062E170E0AD
:104C700080EA90E00E94702CCBE3D1E068817981DA
:104C800028E03CEF4EE150E080E090E00E94BF2A37
:104C90000E9464232A813B81215031094881598136
:104CA0004B505109A12CB12C6BE7C62E65E2D62ED4
:104CB000E12C01E068E171E08AE090E00E94CB2AFB
:104CC0001092230660911F067091200680912106A4
:104CD000909122060E94DC2C8FE095E00E94F22544
:104CE00070E8E72E0BE715E22FEF3FEF41E064E2BB
:104CF00071E084E190E00E94F12BCDB7DEB7EAE0ED
:104D00000C946435EF920F931F938BE795E20E940A
:104D1000FA298AE090E090932206809321069093EE
:104D2000200680931F0646E050E060E371E00E9499
:104D3000F82980911F06909120060E94F92910926F
:104D4000230660911F0670912006809121069091A4
:104D500022060E94DC2C8FE095E00E94F22580E87C
:104D6000E82E0BE715E22FEF3FEF41E062E170E044
:104D70008AE090E00E94F12B81E080930F0284E0B2
:104D80008093210280E090E01F910F91EF900895B1
:104D900060E00E947C250895A2E2B0E0E2EDF6E238
:104DA0000C944D358C01F62E82E28F1588F442E288
:104DB00050E0B801CE0101960E94F23760E0CE01CA
:104DC00001960E947C258EEDF80E0E5D1F4FECCFF4
:104DD00060E0C8010E947C25A296E5E00C9469354C
:104DE000A0E0B0E0E6EFF6E20C944A3580911D06B3
:104DF00090911E068D9768E170E00E94A034C091EA
:104E00001E02D0911F022A97C60FD71F61E0CE0164
:104E10000E94DE188091B80584FF67C0E091BE054E
:104E2000F091BF05C080D180E280F380C482D5823A
:104E3000E682F7828091B4048E3209F03FC08091FF
:104E4000B5048E32D9F5C114D104E104F10439F46A
:104E50008FE290E0909343018093420137C060E07D
:104E600080E090E00E94DE18E091BE05F091BF0561
:104E700080819181A281B38184839583A683B78346
:104E800000E010E061E0C8010E94DE18E091BE057C
:104E9000F091BF0580819181A281B381C816D906A6
:104EA000EA06FB0629F4C482D582E682F78206C0B0
:104EB0000F5F1F4F0F3F110529F7F5CF4CE050E072
:104EC00064EB74E082E491E00E94F23710921F02DA
:104ED00010921E0210921D0210921C028FEF9FEF83
:104EE0009093500180934F011CC0E4EBF4E00190DB
:104EF0000020E9F73197BF01645B7440609324069A
:104F000084EB94E00E94CC26D0935001C0934F01D3
:104F100080911E0290911F020A9790931F02809326
:104F20001E020E94EB2061E0CE010E94DE1880E0AC
:104F300090E0CDB7DEB7E8E00C946635EF92FF92D3
:104F40000F931F93CF930E94BF2DC82F0E942D292E
:104F50008EEA91E00E94E83D80933F0181700E94BB
:104F6000A1290E9499299F938F938EE292E09F93AB
:104F70008F9384EB94E09F938F930E94013884EB8E
:104F8000E82E84E0F82E00E010E02FEF3FEF42E043
:104F900062E271E084E190E00E94952C0F900F9006
:104FA0000F900F900F900F90CC2379F08DEB91E044
:104FB0000E94F63D019629F40E946B290E9401226D
:104FC00004C00E943C2E8111F7CFCF911F910F9109
:104FD000FF90EF900895FF920F931F93CF93DF936D
:104FE000F0903F01F0FAFF24F0F810923F01809119
:104FF0002102A0914001B091410175E0879FA00D71
:10500000B11D112460E0262F30E014968C91149786
:1050100090E0FC0132972E173F0714F51296ED91A0
:10502000FC91139774E1679FE00DF11D11247096B8
:1050300005911491E8010397281739077CF48881BA
:1050400082FB442740F950E0CA0101C0880F2A952D
:10505000EAF790913F01892B80933F016F5FD3CF97
:1050600060913F018EEA91E00E94FC3D888182FDC3
:105070000EC080913F018170F81661F16FEF7FEFF4
:105080008DEB91E00E941A3E0E949E2723C0CCE344
:10509000D2E006E911E08EA580FF0EC04C8D5D8D3B
:1050A0006E8D7F8DC8010E940E3E68A579A5C8014E
:1050B00004960E941A3E06C04FEF5FEFBA01C80186
:1050C0000E940E3E68960A5F1F4F82E0CC39D807D7
:1050D00011F7CFCF0E94632080E090E0CDB7DEB71C
:1050E000E5E00C946935A0E0B0E0E9E7F8E20C9463
:1050F00048350E942E2F362F272F60931B06709362
:105100001C0680931D0690931E0680912102A0919B
:105110004001B091410195E0899FA00DB11D11247E
:105120001496AC901497832F922F00911D06109126
:105130001E0640E050E0B12CBA1451F112962D91A8
:105140003C911397240F351FF9013296C590D490E6
:10515000F9013496E590F490F9013696C591D49111
:10516000F901389665917491C816D90668F4CC0D8A
:10517000DD1D8C179D0740F4E016F10628F46E0D36
:105180007F1D0617170738F0B3944C5E5F4FD4CFDE
:1051900080E090E001C0C901CDB7DEB7EAE00C9431
:1051A000643584B1836084B98AB18C6F8AB987B160
:1051B0008F6187B988B18B6088B98FE39CE90197CB
:1051C000F1F700C00000089544988FE59AEE01972A
:1051D000F1F700C00000449A8FE59AEE0197F1F7CD
:1051E00000C0000008959BB19370282F2C7F922B54
:1051F0009BB995B19C7F8370892B85B94198419A61
:10520000089540982FEF89EF90E021508040904022
:10521000E1F700C0000029B193B1409A2C7F892F9B
:105220008370822B0895CF93C82F4298439880E0D3
:105230000E94F3288C2F0E94F328439ACF9108955F
:10524000CF93C82F429A4398892F0E94F3288C2F1E
:105250000E94F328439ACF9108950F931F93CF9301
:10526000DF930E94D1280E94E4282FEF8DEE92E078
:10527000215080409040E1F700C0000006E117E0B7
:10528000F80184913196C591D49181110BC0CE0162
:10529000009769F0EFE9FFE03197F1F700C00000F7
:1052A0000197F6CF0E941329CE010E9420290D5F9D
:1052B0001F4FF7E0023B1F0719F72FEF81EE94E035
:1052C000215080409040E1F700C00000DF91CF9175
:1052D0001F910F91089587E00E94132983E391E0C5
:1052E0000E942029089587E00E94132980E090E021
:1052F0000E9420290895CF9384B18C7F84B98AB10C
:1053000083708AB9429A43980E940129C82F0E944B
:105310000129439A94B1936094B99AB19C6F9AB958
:105320002C2F30E0322F2227A901482BCA01CF9120
:10533000089580E00E9413290E947B290E947B2906
:105340000895882319F0813071F0089580E60E9455
:10535000132980E097EA0E94202981E00E94132906
:1053600080E091E00CC080E60E94132980E097E283
:105370000E94202981E00E94132980E090E00E9491
:1053800020290895A0E0B0E0E8ECF9E20C944A3559
:105390008C01EB016A01790180E50E941329C801A3
:1053A0000E94202981E50E941329C6010E9420291C
:1053B00082E50E941329CE010E94202983E50E94E4
:1053C0001329C7010E94202980E20E941329C801E5
:1053D0000E94202981E20E941329CE010E942029E7
:1053E00082E20E941329CDB7DEB7E8E00C9466355F
:1053F00008950895CF92DF92EF92FF92CF93DF93BB
:10540000EC0120915101309152012150310940911C
:105410005301509154014150510960E070E080E027
:1054200090E00E94C229C12C8CE2D82EEE24E39495
:10543000F12CCE010E94202981E0C81AD108E10890
:10544000F108B9F7DF91CF91FF90EF90DF90CF9007
:105450000895CF92DF92EF92FF920F931F93DA019C
:10546000A81BB90B1196F901E61BF70B3196AE9FFD
:105470006001AF9FD00CBE9FD00C1124E12CF12C09
:105480000E94C229C114D104E104F10449F0C80109
:105490000E94202981E0C81AD108E108F108F2CF62
:1054A0001F910F91FF90EF90DF90CF900895CF93D1
:1054B000DF93EA019B01AC010E94C229CE010E9448
:1054C0002029DF91CF910895A0E0B0E0EAE6FAE26A
:1054D0000C9442357C01EB013A0129016A01C81A9A
:1054E000D90A5901A61AB70ACC0CDD1CAA0CBB1CA0
:1054F000A8010E94572AAC14BD04C8F4C6019695B1
:1055000087954501881A990AE614F70449F197FC32
:1055100003C021968C189D088FEFE81AF80A8A0CB0
:105520009B1CA801BE01C7010E94572AEDCFC501EF
:10553000969587954601881A990AC415D50581F074
:1055400097FC05C08FEFE81AF80A8A189B08219685
:105550008C0C9D1CA801BE01C7010E94572AEDCFEB
:10556000CDB7DEB7E0E10C945E350F931F93890150
:105570009A01AC010E94292A1F910F9108950F935F
:105580001F93FB01BA0189019A01AF010E94292AE8
:105590001F910F9108954F925F926F927F928F9219
:1055A0009F92AF92BF92CF92DF92EF920F931F9391
:1055B000CF93DF933C014B01EA012901013021F433
:1055C00086010E94292A16C09601A2010E94B52ACE
:1055D0009601A201B401CE010E94B52A9601A40150
:1055E000BE01C3010E94BF2A9601A201BE01C301F0
:1055F0000E94BF2AEE20A1F0A501B401C3010E94C0
:10560000572AA501B201C3010E94572AA501B4017E
:10561000CE010E94572AA501B201CE010E94572A4D
:10562000DF91CF911F910F91EF90DF90CF90BF90BE
:10563000AF909F908F907F906F905F904F90089564
:10564000ADE0B0E0E6E2FBE20C9440357C013B01CA
:105650005D874C872B8781E090E09C01241B350BF4
:105660003A83298317014B017C836B83270143E035
:1056700050E058874F839E838D832D813E8121503A
:1056800031093A872987CC84DD84C60CD71C3B8539
:10569000313039F59801A601B101C2010E94BF2A3B
:1056A0009801A3018C859D85481B590BB101C2014E
:1056B0000E94BF2A98014B815C81AC84BD84AE0CF2
:1056C000BF1CB50167018C859D85C81AD90AC60122
:1056D0000E94BF2A9801A401B501C6010E94BF2AF9
:1056E00038C0A801B601C1010E94572AA8016B81E8
:1056F0007C81AC84BD84AE0CBF1CC5010E94572ABE
:10570000A801B601C2010E94572AA8016B817C81C1
:1057100067012C853D85C21AD30AC6010E94572A0B
:10572000A801B401C5010E94572AA80153018C8524
:105730009D85A81AB90AB501C1010E94572AA8017E
:10574000B501C2010E94572AA801B401C6010E94F6
:10575000572A29813A8137FF0BC02D813E8149812B
:105760005A818F819885480F591F5A83498316C0E3
:105770002D813E8189859A854C855D85841B950B9D
:10578000880F991F059649815A81480F591F5A83DE
:1057900049838C859D8501979D878C874D815E818E
:1057A0004F5F5F4F5E834D838F8198850296988708
:1057B0008F8391E0491A51084FEF241A340A8B81E4
:1057C0009C8101969C838B8391E0891A91084C857A
:1057D0005D85421753070CF050CF2D96E2E10C94F3
:1057E0005C352F923F924F925F927F928F929F9261
:1057F000AF92BF92CF92DF92EF92FF920F931F93DF
:10580000CF93DF93FC01542E4901411102C055246E
:105810005394852D90E09C018E179F0708F4CF01CB
:1058200043E0220F331F4A95E1F7AB014150510984
:10583000240F351FAC0141505109E5E05E9E400D3B
:10584000511D11240E94C22985E0E89E7001112497
:10585000C12CD12CE0EAEE1AF10822242394312C39
:105860000C2C02C0220C331C0A94E2F7712CA12CE0
:10587000B12CF701EA0DFB1DEE54F84FC491D0E0B6
:10588000C221D321412C209711F0C40101C0C801CD
:105890000E94202943945410F6CF8FEFA81AB80A1B
:1058A000E5E0AE16B10429F773945710E0CF8FEFFF
:1058B000C81AD80AE8E0CE16D10479F6DF91CF9164
:1058C0001F910F91FF90EF90DF90CF90BF90AF901E
:1058D0009F908F907F905F904F903F902F90089572
:1058E000A0E0B0E0E6E7FCE20C9441356C015B011E
:1058F000342E4901380186E0489F20011124F70128
:10590000E490EF012196EE2059F083019401432D9C
:10591000B501C6010E94F12BC40CD51CFE01F0CFCD
:10592000CDB7DEB7E1E10C945D35A0E0B0E0EBE986
:10593000FCE20C9441353C016B01342E59014801C5
:1059400086E0489F20011124E701E9908401950138
:10595000432DB601C3010E94F12B640C751C888194
:105960008052803690F3CDB7DEB7E1E10C945D351F
:10597000A0E0B0E0EEEBFCE20C944035EC015B0102
:10598000D42E4901380186E0489F100111242701D7
:10599000F201E1902F01830194014D2DB501CE015B
:1059A0000E94F12BC20DD31DCA94C110F1CFCDB707
:1059B000DEB7E2E10C945C359093280680932706CD
:1059C00070932606609325060895EF92FF920F9339
:1059D0001F93CF93C82F80912506909126067901B9
:1059E0008A019B014C2FBC018091270690912806CB
:1059F0000E94702C80912506909126062CE0C29F73
:105A0000800D911D11249093260680932506CF9139
:105A10001F910F91FF90EF900895EF92FF920F93D7
:105A20001F93CF93C82F8091250690912606790168
:105A30008A019B014C2FBC0180912706909128067A
:105A40000E94952C80912506909126062CE0C29FFD
:105A5000800D911D11249093260680932506CF91E9
:105A60001F910F91FF90EF900895A0E0B0E0EBE35D
:105A7000FDE20C944635FC01EB015901261B370B66
:105A8000DA01A81BB90B0E940F356B017C0195014F
:105A90002150310941505109BE01CF010E94C22954
:105AA000E801812C912C54018C149D04AE04BF0498
:105AB00061F0FE01859194910E9420298FEF881A50
:105AC000980AA80AB80A2296EFCFCDB7DEB7ECE065
:105AD0000C946235E0912E06F0912F0681E090E063
:105AE0009C0100902B0602C0220F331F0A94E2F79C
:105AF000322F3095418134233183E0912E06F0918D
:105B00002F063281232B228338B1AC01009030065E
:105B100002C0440F551F0A94E2F7242F2095232337
:105B200028B937B1AC010090290602C0440F551FB7
:105B30000A94E2F7242F2095232327B938B1AC012A
:105B40000090290602C0440F551F0A94E2F7242F43
:105B50002095232328B9E0912C06F0912D06009082
:105B60002A0602C0880F991F0A94E2F78095928155
:105B70008923828385E38A95F1F70000089587E8F9
:105B800080937A0086EB91E00E94E83D8F3F31F1EF
:105B90008093290685EB91E00E94E83D80932B06D7
:105BA00082EB91E00E94E83D80932A068FEA91E023
:105BB0000E94E83D8093300683EB91E00E94F63D21
:105BC00090932F0680932E0680EB91E00E94F63D85
:105BD00090932D0680932C0681E0089580E008952F
:105BE00048B181E090E09C010090290602C0220F9C
:105BF000331F0A94E2F7242B28B948B19C01009086
:105C0000300602C0220F331F0A94E2F7242B28B972
:105C1000E0912E06F0912F069C0100902B0602C009
:105C2000220F331F0A94E2F73181232B218347B1DE
:105C30009C010090300602C0220F331F0A94E2F745
:105C4000242B27B947B19C010090290602C0220FDE
:105C5000331F0A94E2F7242B27B9E0912C06F09128
:105C60002D0600902A0602C0880F991F0A94E2F7B9
:105C70009181892B81830895CF93DF93F8940E94BB
:105C80006A2DE0912E06F0912F06C081D0E00090A1
:105C90002B0602C0D595C7950A94E2F7C170DD279F
:105CA00081E0C8270E94F02D78948C2FDF91CF914E
:105CB0000895E0912E06F0912F0620912B06409139
:105CC0003006882309F45BC081E090E0BC0102C08B
:105CD000660F771F2A95E2F79B01209531813223C9
:105CE0003183E0912E06F0912F0632812323228307
:105CF00057B19C0101C0220F4A95EAF7252B27B91D
:105D000038B1AC010090300602C0440F551F0A9410
:105D1000E2F7242F2095232328B937B1AC01009056
:105D2000290602C0440F551F0A94E2F7242F20953C
:105D3000232327B938B1AC010090290602C0440FD3
:105D4000551F0A94E2F7242F2095232328B9E091C8
:105D50002C06F0912D0600902A0602C0880F991F8C
:105D60000A94E2F79181982B9183E0912C06F091AF
:105D70002D069281892B8283809129065AC081E069
:105D800090E0BC0102C0660F771F2A95E2F79B01E5
:105D90003181322B3183E0912E06F0912F06209530
:105DA00032812323228337B1BC0102C0660F771FE3
:105DB0004A95E2F7262F2095232327B938B1AC0165
:105DC0000090300602C0440F551F0A94E2F7242FBA
:105DD0002095232328B947B19C010090290602C0D1
:105DE000220F331F0A94E2F7242B27B948B19C01F4
:105DF0000090290602C0220F331F0A94E2F7242BD9
:105E000028B9E0912C06F0912D0600902A0602C0D8
:105E1000880F991F0A94E2F78095918198239183C6
:105E2000E0912C06F0912D06928189238283809146
:105E30003006806480937C0072E07A95F1F700C0B0
:105E400080917A00806480937A0080917A0086FD48
:105E5000FCCF80917800909179000895A8E0B0E09F
:105E6000E4E3FFE20C944035F894409053015090E5
:105E70005401612C712C89EB91E00E94F63D8C015C
:105E80008DEB91E00E94F63D6C01E12CF12C80E05D
:105E90000E94592E98878F838090510190905201D3
:105EA000940140E050E029833A834B835C8387EB85
:105EB00091E00E94F63D9E838D838BEB91E00E94E2
:105EC000F63D4C01A12CB12C81E00E94592E1C0101
:105ED0000E94F02D78944F815885CA01A0E0B0E06F
:105EE0009C01AD012C193D094E095F09C301B201A6
:105EF0000E94843420E030E0A90198012C193D096A
:105F00004E095F090E94EA346901C101A0E0B0E0D6
:105F10009C01AD01281939094A095B0969817A8117
:105F20008B819C810E948434AD81BE818D0120E0F3
:105F300030E0A9019801281939094A095B090E9432
:105F4000EA347901C701B6012896E2E10C945C3588
:105F50000F931F93CF93DF93F89480E00E94592E04
:105F60008C0181E00E94592EEC010E94F02D789462
:105F7000B801CE01DF91CF911F910F910895CF927B
:105F8000DF92EF92FF92CF93DF9320E330E040E087
:105F900050E0BA0180E00E94E61A8091B404813496
:105FA00009F05EC08091B504843509F059C0809134
:105FB000B604883309F054C08091B704883509F0DD
:105FC0004FC08091B8049091B904019709F048C07E
:105FD0008091BA049091BB04019709F041C080916F
:105FE000C604813011F092E101C09AE19093350628
:105FF000823019F080E890E002C080E091E0909358
:10600000340680933306C090D004D090D104E09041
:10601000D204F090D304C7E3D6E020E230E0B70129
:10602000A60180E00E94E61A892B29F480913306AC
:106030009091340617C0C992D992E992F992809151
:10604000B4049091B504A091B604B091B704C80E01
:10605000D91EEA1EFB1E86E0CF3DD807F1F6E6CF3B
:1060600080E090E0DF91CF91FF90EF90DF90CF90B4
:106070000895A0E1B0E0EFE3F0E30C944035FB01BC
:10608000588B4F87019798878F8380913506282FEB
:1060900030E03A8729878F819885B9010E94A03422
:1060A00001E0060F80E1AF85B8898C9380913306BB
:1060B00090913406918380830E946B32EFE4F2E387
:1060C0003197F1F700C0000080913606081761F1A2
:1060D000E02EE81AE7FCE194C12CD12C0E2C000C28
:1060E000FF08CE14DF0498F40E946B32882329F055
:1060F00087EE91EC0197F1F704C0AFECB2E5119790
:10610000F1F700C00000BFEFCB1ADB0AEACF0E9414
:106110006B32882349F0EFEFF3EF21E0E150F040DC
:106120002040E1F700C00000009336060E94643270
:106130006C0110E001501109A801440F551F440FD4
:10614000551F5E834D83FA01E95CF94F8080918091
:10615000A280B38081149104A104B10419F4E12C4C
:10616000F12C92C120E230E0B501A40180E00E9450
:10617000E61A8091BC0490E00817190781F7209077
:10618000BE043090BF042114310449F38091C80447
:106190009091C904A091CA04B091CB04880E991EB5
:1061A000AA1EBB1E28E030E0B501A40180E00E94D9
:1061B000E61A8091B4049091B504A091B604B09110
:1061C000B704880E991EAA1EBB1EC10123E0880FCA
:1061D000991F2A95E1F7A5019401281B390B410964
:1061E00051092B873C874D875E8734E03C8300E074
:1061F00010E01B82812C912C5401E12CF12C4B845A
:106200005C846D847E841A82198228E030E0B301B8
:10621000A20180E00E94E61A892B09F44EC0209169
:10622000B50424FD45C08F81988569857A850E94D3
:10623000A0348F5F9091B40489133AC08091B60462
:106240009091B704AC014C195D090115110571F06D
:10625000141615061CF417FD09C005C0411551059B
:1062600039F117FF25C04017510714F590933206F6
:106270008093310622FD04C0AF85B8892C9305C0F8
:10628000822F8260EF85F8898083AF85B8898C91F1
:1062900086FF03C0BB81BF5FBB838090B804909032
:1062A000B904A090BA04B090BB048A01E980FA80D6
:1062B000E8E04E0E511C611C711C29813A812F5F50
:1062C0003F4F3A8329832216330609F09ECFAF85CC
:1062D000B8898C91811114C0809131069091320659
:1062E0009093B5058093B405EF85F88980818F7709
:1062F00089838083FB81F11115C00FEF1FEF54C01C
:106300000E9464329C0186549A498B3B45E694076F
:1063100008F0C9010E944E325C8151505C835111DA
:106320006ECFDACFED81FE81E95CF94F408051807C
:10633000628073808091C8049091C904A091CA04BE
:10634000B091CB04480E591E6A1E7B1E0FEF1FEF43
:1063500028E030E0B301A20180E00E94E61A4091FB
:10636000B4045091B5046091B6047091B70441151E
:1063700051056105710599F08091B90490E0E81626
:10638000F90641F48091B804803121F40091BA04F7
:106390001091BB04440E551E661E771ED9CFAF85E3
:1063A000B8898C918F7B8C9381149104A104B104E2
:1063B000A1F02091330630913406ED81FE81E95C35
:1063C000F94F4081518162817381480D591D6A1DC9
:1063D0007B1D80E00E94E61A7C018981882311F0F0
:1063E000E12CF12C17FF0AC0809131069091320602
:1063F000C816D906E0F086549A4919C0D801AC54A1
:10640000BB4F5D0100E011E020913306309134066E
:10641000C501845B94408217930730F70E94D337FD
:10642000B8010E94B434F50181935F01EDCF9C0166
:106430002C193D098AEB95E6B1010E94A034C20EE9
:10644000D31EFBEBCF16F5E6DF0620F02AEBC21ACF
:1064500025E6D20ACB018C0D9D1D8B3B35E69307BB
:1064600010F08A5B95460E944E320E946B32882360
:1064700029F08FE39FE10197F1F704C0AFE3BFE19B
:106480001197F1F700C00000EF85F88980818095B1
:106490008083C7016096E2E10C945C352091840012
:1064A00030918500369527958217930718F4B19A95
:1064B000B19BFECF209184003091850036952795C1
:1064C00028173907B8F308958091840090918500CA
:1064D00096958795089580913F0183FB882780F9E1
:1064E00008952091E1063091E2063695279540E027
:1064F00050E060E472E48FE090E00E94C834C9018B
:1065000001970E94611F08958F929F92AF92BF9250
:10651000EF92FF920F931F93CF93DF93EC014C0107
:10652000A12CB12CE091BE05F091BF0542895389A1
:106530006489758984169506A606B70608F05CC0BE
:10654000415051096109710997E076956795579512
:1065500047959A95D1F74F5F5F4F6F4F7F4F7F936E
:106560006F935F934F93CE01880F892F881F990BEC
:10657000919501969F938F938BEC99E09F938F93C6
:1065800084EB94E09F938F930E94013834EBE32EC9
:1065900034E0F32E0AE812E520EE3FEF42E064E833
:1065A00070E083E290E00E94952C20E830E0B50195
:1065B000A40180E00E94E61AE4E3F5E02DB73EB7BF
:1065C000265F3F4F0FB6F8943EBF0FBE2DBF34E09D
:1065D000E43BF30719F092919383F9CF87FD06C04E
:1065E0009AEF9093B6048093360503C09CEF909386
:1065F000B604C80FD11D18C085ECE82E89E0F82E2E
:106600000AE812E520EE3FEF42E064E870E083E242
:1066100090E00E94702C83E890E00E94E3058EEFEA
:106620008093B604C0E0D0E085E58093B404809305
:10663000B50463E870E084EB94E00E94811F63E896
:1066400070E084EB94E00E94521F0E947A1F8FEF4B
:1066500095EA2EE0815090402040E1F700C0000014
:10666000CE01DF91CF911F910F91FF90EF90BF90DE
:10667000AF909F908F90089528E030E040E050E088
:10668000BA0180E00E94E61A9091B4048091B705A7
:10669000963471F49091B504953551F49091B60407
:1066A0009A3431F49091B704993411F4826001C0A6
:1066B0008D7F8093B7058091B70582FF03C088EE78
:1066C00093E002C088E592E09093E2068093E106B1
:1066D0000E9471321092E0061092DF060895A0E049
:1066E000B0E0E5E7F3E30C9444356C014601A12CDE
:1066F000B12CE091BE05F091BF0582899389A489F0
:10670000B58988169906AA06BB0608F045C028E098
:1067100030E0B501A40180E00E94E61AC091B804FF
:10672000D091B9048091B4048436B1F48091B50459
:10673000813671F58091B604843751F58091B704A4
:10674000813631F58091DF069091E00601969093B5
:10675000E0068093DF0620C08236D1F48091B50434
:106760008136B1F48091B604853791F48091B704F5
:10677000843671F48091B70582FDB8CF8091BA0458
:106780009091BB049093E2068093E1060E947132DF
:106790002896CC0EDD1EAACF84EB94E06090BA045C
:1067A0007090BB04C091B804D091B9047F926F92ED
:1067B000DF93CF932091E2062F932091E1062F9350
:1067C00025EA39E03F932F939F938F930E940138DE
:1067D00094EBE92E94E0F92E0AE812E520EE37E07A
:1067E00041E069E970E08FE090E00E94952C8DB760
:1067F0009EB70A960FB6F8949EBF0FBE8DBFC30119
:10680000009741F0EFE9FFE03197F1F700C0000099
:106810000197F6CFE091BE05F091BF05828993897B
:10682000A489B58988169906AA06BB0608F064C033
:106830008091E0068F938091DF068F9387E999E03E
:106840009F938F9384EB94E09F938F930E940138E2
:1068500084EBE82E84E0F82E0AE812E520EE3FEF04
:1068600042E064E870E083E290E00E94952C8601AB
:10687000085F1F4F0F900F900F900F900F900F9089
:10688000DD24D39480E091E0209731F1C130F1E034
:10689000DF0720F05E01BA94EC0102C0A12CB12CFC
:1068A000A80160E070E09E0180E00E94E61A080FF7
:1068B000191FBE0184EB94E00E94811FDD2041F08E
:1068C0008091B6048E3F21F41092E0061092DF060C
:1068D000D12CCE01E501D8CF8091DF069091E00662
:1068E000892B61F48FEF93ECE9E081509040E04018
:1068F000E1F700C0000002C000E010E0C801CDB721
:10690000DEB7EEE00C946035DB018F939F930E941D
:106910002D35BF91AF91A29F800D911DA39F900D2A
:10692000B29F900D11240895991B79E004C0991F1E
:10693000961708F0961B881F7A95C9F780950895D9
:10694000AA1BBB1B51E107C0AA1FBB1FA617B70795
:1069500010F0A61BB70B881F991F5A95A9F78095B1
:106960009095BC01CD01089597FB072E16F4009475
:1069700007D077FD09D00E94A03407FC05D03EF473
:10698000909581959F4F0895709561957F4F0895DB
:10699000A1E21A2EAA1BBB1BFD010DC0AA1FBB1F23
:1069A000EE1FFF1FA217B307E407F50720F0A21B95
:1069B000B30BE40BF50B661F771F881F991F1A9402
:1069C00069F760957095809590959B01AC01BD012C
:1069D000CF010895052E97FB1EF400940E94013507
:1069E00057FD07D00E94C83407FC03D04EF40C9426
:1069F000013550954095309521953F4F4F4F5F4F52
:106A0000089590958095709561957F4F8F4F9F4F1A
:106A10000895EE0FFF1F0590F491E02D09940E9458
:106A20001735332312F48A1B9B0B0C942835A29F35
:106A3000B001B39FC001A39F700D811D1124911D52
:106A4000B29F700D811D1124911D08950E9417356C
:106A5000B7FF0895821B930B08950E941735A59FD9
:106A6000900DB49F900DA49F800D911D1124089549
:106A7000B7FF0C942D350E942D35821B930B089582
:106A80002F923F924F925F926F927F928F929F923E
:106A9000AF92BF92CF92DF92EF92FF920F931F932C
:106AA000CF93DF93CDB7DEB7CA1BDB0B0FB6F894DD
:106AB000DEBF0FBECDBF09942A88398848885F841D
:106AC0006E847D848C849B84AA84B984C884DF808E
:106AD000EE80FD800C811B81AA81B981CE0FD11D72
:106AE0000FB6F894DEBF0FBECDBFED01089550582C
:106AF000BB27AA270E948F350C94E0360E94D2361D
:106B000038F00E94D93620F039F49F3F19F426F46A
:106B10000C94CF360EF4E095E7FB0C94C936E92FC0
:106B20000E94F13658F3BA17620773078407950776
:106B300020F079F4A6F50C9413370EF4E0950B2EA3
:106B4000BA2FA02D0B01B90190010C01CA01A001BF
:106B50001124FF27591B99F0593F50F4503E68F11A
:106B60001A16F040A22F232F342F4427585FF3CF5B
:106B7000469537952795A795F0405395C9F77EF42C
:106B80001F16BA0B620B730B840BBAF09150A1F075
:106B9000FF0FBB1F661F771F881FC2F70EC0BA0FFB
:106BA000621F731F841F48F4879577956795B79583
:106BB000F7959E3F08F0B0CF9395880F08F099277E
:106BC000EE0F9795879508950E94F8350C94E0365E
:106BD0000E94D93658F00E94D23640F029F45F3F27
:106BE00029F00C94C93651110C9414370C94CF36FB
:106BF0000E94F13668F39923B1F3552391F3951B65
:106C0000550BBB27AA2762177307840738F09F5FCD
:106C10005F4F220F331F441FAA1FA9F335D00E2E3A
:106C20003AF0E0E832D091505040E695001CCAF7A7
:106C30002BD0FE2F29D0660F771F881FBB1F26176A
:106C400037074807AB07B0E809F0BB0B802DBF0141
:106C5000FF2793585F4F3AF09E3F510578F00C9410
:106C6000C9360C9414375F3FE4F3983ED4F386950D
:106C700077956795B795F7959F5FC9F7880F911D31
:106C80009695879597F90895E1E0660F771F881F1D
:106C9000BB1F621773078407BA0720F0621B730BD0
:106CA000840BBA0BEE1F88F7E09508950E945D36BD
:106CB0006894B1110C94143708950E94F93688F045
:106CC0009F5798F0B92F9927B751B0F0E1F0660FB0
:106CD000771F881F991F1AF0BA95C9F714C0B130F1
:106CE00091F00E941337B1E008950C941337672F89
:106CF000782F8827B85F39F0B93FCCF38695779520
:106D00006795B395D9F73EF4909580957095619508
:106D10007F4F8F4F9F4F0895E89409C097FB3EF433
:106D200090958095709561957F4F8F4F9F4F9923D8
:106D3000A9F0F92F96E9BB279395F6958795779556
:106D40006795B795F111F8CFFAF4BB0F11F460FF16
:106D50001BC06F5F7F4F8F4F9F4F16C0882311F06E
:106D600096E911C0772321F09EE8872F762F05C082
:106D7000662371F096E8862F70E060E02AF09A951D
:106D8000660F771F881FDAF7880F9695879597F912
:106D9000089597F99F6780E870E060E008959FEF9D
:106DA00080EC089500240A941616170618060906A2
:106DB000089500240A941216130614060506089571
:106DC000092E0394000C11F4882352F0BB0F40F4F9
:106DD000BF2B11F460FF04C06F5F7F4F8F4F9F4F39
:106DE000089557FD9058440F551F59F05F3F71F0BB
:106DF0004795880F97FB991F61F09F3F79F0879522
:106E00000895121613061406551FF2CF4695F1DFAA
:106E100008C0161617061806991FF1CF869571053A
:106E2000610508940895E894BB2766277727CB016E
:106E300097F908950E942D370C94E0360E94D236BF
:106E400038F00E94D93620F0952311F00C94C93601
:106E50000C94CF3611240C9414370E94F13670F341
:106E6000959FC1F3950F50E0551F629FF001729FEF
:106E7000BB27F00DB11D639FAA27F00DB11DAA1FFE
:106E8000649F6627B00DA11D661F829F2227B00D4B
:106E9000A11D621F739FB00DA11D621F839FA00DD6
:106EA000611D221F749F3327A00D611D231F849F26
:106EB000600D211D822F762F6A2F11249F5750407D
:106EC0009AF0F1F088234AF0EE0FFF1FBB1F661FF8
:106ED000771F881F91505040A9F79E3F510580F0C1
:106EE0000C94C9360C9414375F3FE4F3983ED4F306
:106EF000869577956795B795F795E7959F5FC1F765
:106F0000FE2B880F911D9695879597F908958F927E
:106F10009F92AF92BF92CF92DF92EF92FF92CF9368
:106F2000DF93EC01688179818A819B81611571050C
:106F30008105910521F464E279ED8BE597E02DE17F
:106F400033EF41E050E00E94EA3449015A019B01CD
:106F5000AC01A7EAB1E40E942D356B017C01ACEED7
:106F6000B4EFA50194010E943B35DC01CB018C0DEF
:106F70009D1DAE1DBF1DB7FF03C00197A109B048FD
:106F800088839983AA83BB839F77DF91CF91FF90FA
:106F9000EF90DF90CF90BF90AF909F908F9008952B
:106FA0000E948737089585E591E00E94873708950C
:106FB000A0E0B0E08093550190935601A093570153
:106FC000B09358010895FB01DC014150504048F056
:106FD00005900D920020C9F701C01D92415050400C
:106FE000E0F70895FB01DC014150504048F001906A
:106FF0000D920020C9F701C01D9241505040E0F7AA
:107000000895AEE0B0E0E7E0F8E30C944E350D896A
:107010001E898EE08C831A8309838FEF9FE79E83FE
:107020008D83AE01475E5F4F6F89788DCE010196EB
:107030000E943C38EF81F885E00FF11F10822E96F8
:10704000E4E00C946A35AEE0B0E0E9E2F8E30C94D9
:1070500050358DE08C838B899C899A838983AE011E
:10706000495E5F4F6D897E89CE0101960E94B93BD2
:107070002E96E2E00C946C35ABE0B0E0E2E4F8E38D
:107080000C9440356C017B018A01FC011782168249
:10709000838181FFCCC1CE0101963C01F601938131
:1070A000F70193FD859193FF81917F01882309F476
:1070B000BAC1853239F493FD859193FF81917F01A7
:1070C000853229F4B60190E00E94323DE7CF912C41
:1070D000212C312CFFE1F315D8F08B3279F038F404
:1070E000803279F08332A1F4232D20611DC08D32CE
:1070F00061F0803369F4232D216016C0832D8260F6
:10710000382EE32DE4603E2E2AC0F32DF8601DC01A
:1071100037FC2DC020ED280F2A3040F08E32B9F414
:1071200036FC81C1232D2064322E19C036FE06C0E4
:107130008AE0989E200D1124922E11C0EAE02E9E26
:10714000200D1124222EF32DF0623F2E08C08C3624
:1071500021F4832D8068382E02C0883641F4F7016F
:1071600093FD859193FF81917F018111B3CF982F7A
:107170009F7D9554933028F40C5F1F4F9FE39983B4
:107180000DC0833631F0833771F0833509F059C073
:1071900021C0F801808189830E5F1F4F882483946A
:1071A000912C530113C02801F2E04F0E511CF8013D
:1071B000A080B18036FE03C0692D70E002C06FEF81
:1071C0007FEFC5010E94E93C4C018201F32DFF775E
:1071D0003F2E16C0280122E0420E511CF801A0806B
:1071E000B18036FE03C0692D70E002C06FEF7FEF03
:1071F000C5010E94DE3C4C01F32DF0683F2E820158
:1072000033FC1BC0822D90E088169906B0F4B601BD
:1072100080E290E00E94323D2A94F4CFF50137FCE1
:10722000859137FE81915F01B60190E00E94323D69
:1072300021102A9421E0821A91088114910471F797
:10724000E8C0843611F0893641F5F80137FE07C0F1
:1072500060817181828193810C5F1F4F08C06081C2
:107260007181072E000C880B990B0E5F1F4FF32DB9
:10727000FF763F2E97FF09C0909580957095619598
:107280007F4F8F4F9F4FF0683F2E2AE030E0A301E1
:107290000E94873D882E861845C0853731F4232DFE
:1072A0002F7EB22E2AE030E025C0932D997FB92E93
:1072B0008F36C1F018F4883579F0B5C0803719F0F1
:1072C000883721F0B0C0E92FE061BE2EB4FE0DC0BA
:1072D000FB2DF460BF2E09C034FE0AC0292F2660A2
:1072E000B22E06C028E030E005C020E130E002C048
:1072F00020E132E0F801B7FE07C060817181828130
:1073000093810C5F1F4F06C06081718180E090E027
:107310000E5F1F4FA3010E94873D882E8618FB2D0C
:10732000FF773F2E36FE0DC0232D2E7FA22E89140F
:1073300058F434FE0BC032FC09C0832D8E7EA82E7B
:1073400005C0B82CA32C03C0B82C01C0B92CA4FED6
:107350000FC0FE01E80DF11D8081803321F49A2DCC
:10736000997EA92E09C0A2FE06C0B394B39404C0AE
:107370008A2D867809F0B394A3FC11C0A0FE06C044
:10738000B21488F4280C922C9B180EC0B21460F42E
:10739000B60180E290E00E94323DB394F7CFB21480
:1073A00018F42B1802C0982C212CA4FE10C0B60192
:1073B00080E390E00E94323DA2FE17C0A1FC03C012
:1073C00088E790E002C088E590E0B6010CC08A2D05
:1073D000867859F0A1FE02C08BE201C080E2A7FCD2
:1073E0008DE2B60190E00E94323D891438F4B60176
:1073F00080E390E00E94323D9A94F7CF8A94F301A3
:10740000E80DF11D8081B60190E00E94323D8110AF
:10741000F5CF222009F442CEB60180E290E00E942E
:10742000323D2A94F6CFF6018681978102C08FEF14
:107430009FEF2B96E2E10C945C3520FD09C0FC0126
:1074400023FD05C022FF02C0738362835183408302
:10745000089544FD17C046FD17C0AB01BC01DA0119
:10746000FB01AA0FBB1FEE1FFF1F1094D1F74A0F9D
:107470005B1F6E1F7F1FCB01BA01660F771F881F2E
:10748000991F09C033E001C034E0660F771F881FE1
:10749000991F3150D1F7620F711D811D911D089503
:1074A0000F931F93CF93DF938C01C8010E94F43C8C
:1074B000EC0197FD08C00E94CA3C892BB1F7B801C6
:1074C000CE010E946E3DCE01DF91CF911F910F91B1
:1074D00008958F929F92AF92BF92EF92FF920F9377
:1074E0001F93CF93DF938C01D62F7A01B22E0E9487
:1074F000F43C9C0133272B32310531F02D3231051C
:1075000061F48B2D8068B82ED15011F480E068C0F2
:10751000C8010E94F43C97FDF9CFCB2DCD7F2B2DD8
:10752000207309F58033F9F4AA24AA94AD0E09F466
:1075300043C0C8010E94F43C97FD3EC09C012F7DD2
:1075400033272835310549F4C264D250A9F1C80166
:107550000E94F43C97FF07C02FC0B6FE02C0C26075
:1075600001C0C261DA2D812C912C540120ED280F2D
:10757000283080F0C4FF04C0B8010E946E3D19C0DD
:107580002A3040F0C6FFF8CF2F7D3FEE320F363065
:1075900098F727504C2FC501B4010E94293A4B019E
:1075A0005C01C260D15059F0C8010E94F43C97FFC1
:1075B000DDCFC1FD04C0AACF812C912C5401C7FF9F
:1075C00008C0B094A09490948094811C911CA11C3C
:1075D000B11C2C2FB501A401C7010E941D3A81E006
:1075E000DF91CF911F910F91FF90EF90BF90AF90DF
:1075F0009F908F900895A0E2B0E0E1E0FBE30C944F
:1076000043355C01962E7A01F9018E010F5F1F4F01
:10761000680180E2D8011D928A95E9F7D501139699
:107620008C9080E090E0612C712C30E061E070E0A3
:1076300083FC259183FE21918F01522E211103C0DD
:1076400080E090E092C02E3511F4009751F1432F65
:1076500050E0481759073CF42D3559F12D3219F4F3
:10766000772009F103C0772009F46AC0452D4695BB
:1076700046954695D601A40FB11D452D47708B0147
:1076800002C0000F111F4A95E2F7A8015C91452B3B
:107690004C93651459F0561410F45394E7CF5A9450
:1076A000E5CF31E004C07724739401C0712C0196BA
:1076B000BFCF772019F08E8180628E83311103C095
:1076C0008824839417C0F6019E012F5D3F4F80816F
:1076D000809581932E173F07D1F7F2CFE114F10483
:1076E00029F0D7018C93F70131967F019A94812C70
:1076F0009920F9F0C5010E94F43C97FD18C0FC01E7
:10770000FF2723E0F595E7952A95E1F7EC0DFD1DA0
:10771000208130E0AC014770552702C03595279590
:107720004A95E2F720FDDACFB5010E946E3D811047
:1077300087CFE114F10411F0D7011C92C80115C0E4
:10774000422F469546954695D601A40FB11D422F6E
:1077500047708B0102C0000F111F4A95E2F7A80184
:107760005C91452B4C93622EA2CFA096EFE00C9437
:107770005F35A0E0B0E0EFEBFBE30C9443356C0128
:10778000EB015A01FC0117821682512CF601E380AD
:10779000FE01E3FC8591E3FE8191182FEF01882320
:1077A00009F4EEC090E00E94CA3C892B21F0C6018A
:1077B0000E94503AEBCF153241F4FE01E3FC1591E3
:1077C000E3FE1191EF01153281F4C6010E94F43CF1
:1077D00097FDD4C0412F50E09C0133272417350773
:1077E000A9F2B6010E946E3DCBC01A3239F4E3FC17
:1077F0001591E3FE1191EF0101E001C000E0F12CD1
:1078000020ED210F2A3080F402606F2D70E080E0BF
:1078100090E040E20E94293AF62EFE01E3FC159129
:10782000E3FE1191EF01ECCF01FF03C0F11003C0A3
:10783000A7C0FF24FA94183619F01C3651F010C076
:10784000FE01E3FC1591E3FE1191EF01183641F4BE
:1078500008600460FE01E3FC1591E3FE1191EF0165
:10786000112309F48DC0612F70E088EE90E00E9432
:10787000D33C892B09F484C000FD07C0F50180804A
:107880009180C50102965C0102C0812C912C1E36AC
:1078900051F4F6014681578160E070E0202FC40169
:1078A0000E941D3A73CF1336A9F401FD02C0FF24D4
:1078B000F394C6010E94F43C97FD60C081149104CA
:1078C00029F0F4018083C40101964C01FA94F1106F
:1078D000F0CF50C01B3559F49E01A4016F2DC60195
:1078E0000E94FB3AEC01892B09F044C03EC0C6015E
:1078F0000E94503A97FD42C01F3661F128F41436B9
:1079000039F1193651F128C0133771F0153701F1EB
:1079100023C08114910429F0F4016082C40101960E
:107920004C01FA94FF2071F0C6010E94F43C3C0126
:1079300097FD08C00E94CA3C892B59F3B601C301C8
:107940000E946E3D81149104A9F0F401108212C0CE
:10795000006203C0006101C00064202FA4016F2DEC
:10796000C6010E94693A811105C0F60183818073C6
:1079700029F406C000FD0ACF539408CF552019F012
:10798000852D90E002C08FEF9FEFCDB7DEB7EFE01F
:107990000C945F3591110C94E53D803219F08950BB
:1079A0008550C8F70895FC010590061621F00020C7
:1079B000D9F7C00108953197CF010895FC010590D2
:1079C000615070400110D8F7809590958E0F9F1FE1
:1079D0000895FC016150704001900110D8F7809526
:1079E00090958E0F9F1F0895CF93DF93EC012B810D
:1079F00020FF33C026FF0AC02F7B2B838E819F81FF
:107A000001969F838E838A8190E029C022FF0FC058
:107A1000E881F9818081082E000C990B009719F4F8
:107A200020622B831AC03196F983E8830EC0EA8561
:107A3000FB85099597FF09C02B81019611F080E223
:107A400001C080E1822B8B8308C02E813F812F5F94
:107A50003F4F3F832E83992702C08FEF9FEFDF9127
:107A6000CF9108950F931F93CF93DF93FB01238151
:107A700021FD03C08FEF9FEF2CC022FF16C046816F
:107A80005781248135814217530744F4A081B18185
:107A90009D012F5F3F4F318320838C932681378157
:107AA0002F5F3F4F3783268314C08B01EC01FB010E
:107AB0000084F185E02D0995892BE1F6D801169611
:107AC0008D919C911797019617969C938E9316977C
:107AD000CE01DF91CF911F910F910895FB0123817A
:107AE00020FF12C026FD10C08F3F3FEF930761F0CB
:107AF00082832F7D206423832681378121503109A1
:107B000037832683992708958FEF9FEF0895FA0111
:107B1000AA27283051F1203181F1E8946F936E7FCC
:107B20006E5F7F4F8F4F9F4FAF4FB1E03ED0B4E0BD
:107B30003CD0670F781F891F9A1FA11D680F791FFE
:107B40008A1F911DA11D6A0F711D811D911DA11D0F
:107B500020D009F468943F912AE0269F112430191F
:107B6000305D3193DEF6CF010895462F4770405DBA
:107B70004193B3E00FD0C9F7F6CF462F4F70405D69
:107B80004A3318F0495D31FD4052419302D0A9F7C4
:107B9000EACFB4E0A6959795879577956795BA95BE
:107BA000C9F700976105710508959B01AC010A2E84
:107BB00006945795479537952795BA95C9F7620F5B
:107BC000731F841F951FA01D089599278827089566
:107BD000F999FECF92BD81BDF89A992780B5089595
:107BE000A6E1B0E044E050E00C94223EA8E1B0E011
:107BF00042E050E00C94223E262FF999FECF92BD30
:107C000081BDF89A019700B4021639F01FBA20BD61
:107C10000FB6F894FA9AF99A0FBE08950396272F93
:107C20000E94FD3D0E94FC3D252F0E94FD3D242F1A
:107C30000C94FD3D0196272F0E94FD3D0C94FC3DC8
:107C4000DC01CB01FC01F999FECF06C0F2BDE1BD1C
:107C5000F89A319600B40D9241505040B8F708950B
:047C6000F894FFCFC6
:107C64003C02FF2901F62526040A4B249A030799AE
:107C740024FA02082125AA0204822696020101039D
:107C840003030303030303030303030103030303C2
:107C94000303030303030303030307F00040010189
:107CA40005012F000000000000000000000000FF9C
:107CB400FF4001F000010000005374617274005031
:107CC4006175736500547572626F0045786974005C
:107CD400526F74617465005363726F6C6C00426F11
:107CE4006F744431003130353000426C616E6B008A
:107CF40053617665496D005361766500546F700079
:107D040050726576004F4B004E657874004C617379
:107D1400740044303A0044313A3C656D7074793EE5
:107D240020202020200044323A3C656D7074793E56
:107D340020202020200044333A3C656D7074793E45
:107D440020202020200044343A3C656D7074793E34
:107D5400202020202000546170653A004E65770091
:087D64003E3E3E00436667004D
:00000001FF
